:100000006AC30000A0C300009EC300009CC30000A0
:100010009AC3000098C3000096C3000094C3000078
:1000200092C3000090C300000C943B330C94233423
:100030000C94F03288C3000086C3000084C3000023
:1000400082C3000080C300007EC300007CC30000A8
:100050007AC300000C94173376C3000074C3000009
:1000600072C3000070C300006EC300006CC30000C8
:100070006AC3000068C3000066C3000064C30000D8
:1000800062C3000060C300005EC300005CC30000E8
:100090005AC3000058C3000056C3000054C30000F8
:1000A00052C3000050C300004EC300000501090206
:1000B000A10185020901A1000509190129081500FE
:1000C0002501950875018102050109300931158165
:1000D000257F95027508810609381581257F9501D0
:1000E00075088106050C0A38021581257F95017572
:1000F000088106C0C005010980A101850319012AF4
:10010000B700150126B700950175108100C0050CD8
:100110000901A101850419012AA002150126A002E6
:10012000950175108100C005010906A1018506052C
:100130000719E029E71500250195087501810205D9
:1001400007190029EF1500250195F07501810205B9
:10015000081901290595057501910295017503910D
:1001600001C00660FF0961A1010962150026FF00B8
:100170009520750881020963150026FF00952075FA
:10018000089102C005010906A101050719E029E748
:1001900015002501950875018102950175088101F9
:1001A0000507190029FF150026FF0095067508812F
:1001B000000508190129051500250195057501910E
:1001C00002950175039101C00000000000000000CD
:1001D000000000000000000000000000000000001F
:1001E0000000000000000000000000007E0F00D4AE
:1001F000FFFFFFC7000000780000000000000000C3
:100200002A2B280000000000000000000000000071
:1002100000000029000000002C1E3420212224347C
:100220002627252E362D3738271E1F20212223244E
:1002300025263333362E37381F0405060708090AEA
:100240000B0C0D0E0F101112131415161718191A86
:100250001B1C1D2F3130232D350405060708090A04
:100260000B0C0D0E0F101112131415161718191A66
:100270001B1C1D2F3130354C09025B00030100A00F
:10028000FA09040000010301010009211101000124
:10029000224400070581030800020904010002034B
:1002A000000000092111010001222200070582033C
:1002B00020000107050303200001090402000103D7
:1002C00000000009211101000122B6000705840386
:1002D00020000212010002000000086469420000D0
:1002E00001010203011C037600690061006C003A01
:1002F00000660036003400630032006200330063A1
:100300000000001803410062006100630075007383
:10031000002000490044003400320000000E034970
:100320000044004F00420041004F00000004030958
:1003300004167C14001A000800150017001C001891
:10034000000C00120013002A002B00040016000706
:100350000009000A000B000D000E000F000000282D
:1003600000E1001D001B000600190005001100102F
:1003700000E500000052004C00E000E300E2002C29
:100380004200000000777C00000000500051004F48
:100390000035001E001F0020002100220023002441
:1003A00000250026002700010001000000000000D9
:1003B0000000002D002E002F003000310000000151
:1003C0000001000000000033003400360037003820
:1003D00000010000004B0049000100010001002362
:1003E00052000000000100000000004A004E004DD5
:1003F0000029003A003B003C003D003E003F004029
:100400000041004200430001000100000000000024
:10041000000000440045004600470048000000017D
:1004200000010000000000000000000000000000CB
:100430000065000000A900A800E400E700E6000154
:100440000000000000010000000000AD00AA00AEA6
:10045000000100000000000000007C00000000001F
:100460000000000000000001000100207821782435
:10047000782378267825780000000000000000012D
:10048000000100227800000000000000001370004E
:1004900000000000002778000001000100010001B9
:1004A00000000000000100000000002A78287829E0
:1004B00078000101010101010101010202020202B1
:1004C00002020202030303030303030304040404FC
:1004D00004040405050505050606060606070707C4
:1004E000070708080808090909090A0A0A0B0B0B7B
:1004F0000C0C0C0D0D0D0E0E0E0F0F0F1010111118
:10050000111212131314141515161617171818199B
:10051000191A1A1B1B1C1D1D1E1E1F202021222202
:10052000232424252626272829292A2B2C2D2D2E45
:100530002F30313232333435363738393A3B3C3D5F
:100540003E3F404142434445464748494A4C4D4E50
:100550004F50515354555658595A5B5D5E5F616216
:1005600064656668696B6C6D6F7072737577787AA5
:100570007B7D7E8082838587888A8C8E8F91939500
:1005800096989A9C9EA0A2A3A5A7A9ABADAFB1B324
:10059000B5B7BABCBEC0C2C4C6C9CBCDCFD1D4D604
:1005A000D8DBDDDFE2E4E7E9EBEEF0F3F5F8FAFDA6
:1005B000FFFD377A585A000004E6D6B446020021FF
:1005C0000116000000742FE5A3E001F200E45D00D5
:1005D0003D8889C65436C3174FE4E041A5D3C77D93
:1005E0003CE86CEB04785CBC21B59E65D58CFE655F
:1005F000EA780141C14286CDAFBD34EC13B4BFFAF5
:100600000C2FE963ED9F658B1A40DE424491325016
:10061000B6482A00ACD639BB9A4FD5A2BB23DA1F05
:1006200058B11C893F44309CADD94AD59E87AF3024
:10063000786C50CA864C4A65EDC22DD3121E703DAF
:1006400057C252BA73C0D7FAC7D866749B8E3CF3B0
:10065000494DB67CAADA281EB5DF10D685EDF451D7
:10066000F8E5B6F10763331A8AA69A0A0874CD230F
:10067000AF152245975F14F7F7E813CBC865F04A2A
:1006800089C546C1573A575E0FF774F821177FB6F0
:100690008A3B24CFD9986149B924DC04118986BFEB
:1006A0000220804E3701805637CD577D876F8013EB
:1006B0008467158800AC5F02054D0FA4C40001805B
:1006C00002F30300007594B031B1C467FB0200006F
:1006D000000004595A0011241FBECFEFDAE0DEBF3C
:1006E000CDBF04B603FE18C080919A0590919B057A
:1006F000A0919C05B0919D058730904BA740B04BD1
:1007000059F410929A0510929B0510929C05109234
:100710009D05E0E0F8E3099512E0A0E0B1E0E4E532
:10072000FCE602C005900D92AE36B107D9F725E080
:10073000AEE6B2E001C01D92AA39B207E1F70E940D
:10074000412B0C949E355CCC9C01FB019A95811544
:100750009F4120F5832F8170B32FB270AA27732F8A
:1007600074706627532F5870442734FF0DC082954C
:10077000807FAB2B09F08062672B09F08064452BEA
:1007800009F0806809950895AB2B09F08260672B0A
:1007900009F08460452BB1F38860F4CF80E0F2CF9C
:1007A00080939605089580939705089521E030E0A1
:1007B00001C0220F8A95EAF780919705822BF3CF2B
:1007C00021E030E0A90102C0440F551F8A95E2F7ED
:1007D000CA018095909197058923E5CF292F943000
:1007E00090F58C3080F590E03CE0239F800D911DCA
:1007F0001124282F277041E001C0440F2A95EAF701
:1008000023E0969587952A95E1F7FC01EE0FFF1FEF
:10081000E80FF91FE658FB4F20E030E070E05191FF
:10082000DF01CB01022E02C0969587950A94E2F76C
:10083000817081958527842385278E932F5F3F4F75
:100840002330310561F70895292F943078F58C30E5
:1008500068F590E03CE0239F800D911D1124682FE6
:10086000677023E0969587952A95E1F7FC01EE0FD6
:10087000FF1FE80FF91FE658FB4F40E050E080E013
:10088000219130E0062E02C0369527950A94E2F7B2
:1008900021703327042E01C0220F0A94EAF7822B1D
:1008A0004F5F5F4F4330510559F7089580E0089539
:1008B0009091970521E030E0F90101C0EE0F8A9593
:1008C000EAF7D90102C0AA0FBB1F6A95E2F7EA2B2B
:1008D00001C0220F4A95EAF7892F8E23E81303C03F
:1008E000892F822B60CF2095822F8923FBCF809187
:1008F000280490912704981301C008958F5F877092
:10090000FACF9091F704809589238093F704282FDC
:100910002770211110C0891771F09091990592FFED
:100920000AC08695869586954BDF1092F704109243
:10093000F9041092F8040895982F90958091F4048A
:1009400089238093F40408958091F304811531F094
:100950001092F3041092FB041092FA040895803E62
:100960009105D9F1C8F48133910509F482C048F4A6
:100970008932910509F472C08A32910509F480C068
:10098000089589339105E9F082389105D1F08533D6
:10099000910509F45EC00895843E9105D9F148F4AB
:1009A000823E910539F1833E910549F181EE90E057
:1009B0000895863E9105C9F1873E910509F43EC030
:1009C0000895209198052370211164C02091990504
:1009D00023FF14C089E290E008952091980520FD3E
:1009E00045C03091990530FF09C024FD24C083EE35
:1009F00090E008952091980522FDF7CF0895209169
:100A0000980522FD44C03091990530FD43C024FF74
:100A1000F5CF11C02091990521FFF0CF8091980565
:100A200084FD09C087EE90E008952091980523FF8A
:100A3000E5CF24FFF7CF80E090E00895209198055E
:100A400023FD2BC03091990531FFE1CF84EE90E07A
:100A500008952091980525FFD1CFBCCF209198050E
:100A600025FD1EC02091990523FFC8CF89E390E0A2
:100A700008952091980526FFC1CF8AE290E008955D
:100A80002091980526FFBACF81E390E0089582EE89
:100A900090E0089580EE90E0089586EE90E008954D
:100AA00085E390E008959091980592FF10C041E091
:100AB000282F2471243009F040E031E0282F2871DC
:100AC000283009F030E0431711F02CE0822793FF23
:100AD00010C041E0282F2471243109F040E031E0BA
:100AE000282F2871283109F030E0431711F02CE04D
:100AF00082273091990530FF10C051E0282F2171D5
:100B0000213009F050E041E0282F2871283009F009
:100B100040E0541711F029E0822731FF10C041E076
:100B2000282F2171213109F040E031E0282F287170
:100B3000283109F030E0431711F029E0822794FDB5
:100B4000877E08951F93CF93DF9309DFEC01811512
:100B500022E5920708F052C0811540E5940708F09D
:100B6000CDC0803E910520F58D3C910508F0A1C0D7
:100B7000883A910570F4853A910508F097C0813064
:100B80009105B9F10497813A910598F1C0E0D0E060
:100B900030C0885A91094B97C8F7C85AD0E0CC0F9B
:100BA000DD1FCE5FDD4F0990D881C02DD46421C0F8
:100BB000811550E49507B0F4C11580E2D80708F01C
:100BC000B3C0C83ED105A8F0CE019A9581159F41CA
:100BD000E8F68D2F68DF182FCE019927C0DEEC01D3
:100BE000D12B07C09927BBDECC27DF70C82BD92BB0
:100BF000D06ACE01DF91CF911F910895803842E5F0
:100C00009407C8F5803652E5950708F05BC0C034FC
:100C100082E5D807D0F4C03292E5D90708F04BC07E
:100C20008C2F8695869520E2829FC0011124C37087
:100C300021E030E0A90102C0440F551FCA95E2F738
:100C4000EA01C82BD92BDD68D4CF8C2F86958695E9
:100C5000877050E2859FC0011124C37021E030E00D
:100C6000A90102C0440F551FCA95E2F7EA01C82B3B
:100C7000D92BDC68BECF803C52E5950758F48F71C4
:100C8000C03AD245A0F590E0982F8827EC01C46FB8
:100C9000D06AAFCF805C9245809708F077CFDC2F89
:100CA000CC27CC27DF71C06FD06AA3CFA497D064C4
:100CB000A0CFD0659ECFCF71D0E0DC2FCC27C16F05
:100CC000D06A97CF86958695877020E2829FC00173
:100CD0001124C37021E030E0A90102C0440F551F68
:100CE000CA95E2F7EA01C82BD92BDA6882CFDBDE9E
:100CF000C82FD0E0DC2FCC27D0627BCF8F71D3DE22
:100D000093E0CC0FDD1F9A95E1F7CC27DF70282FF9
:100D100030E084FF05C050E1859F90011124332706
:100D2000C22BD32BD06965CF8D2F8F71BCDE182FCE
:100D3000CE01992714DEEC01D12BDECF80E008959F
:100D4000F894E82FE295EF70F0E041A18F7021E078
:100D500030E0B90102C0660F771F8A95E2F7CB0138
:100D6000962F9095942391A392A1892B82A3789496
:100D70000895CF92DF92EF92FF921F93CF93DF936C
:100D8000172FE82FF0E0EF54FB4F71110CC0E491E6
:100D90008E2F7E2F6E2FDF91CF911F91FF90EF90BE
:100DA000DF90CF900895E62EF12CC72ED12CF49130
:100DB000EF2F86E0689F90011124CFEFD0E0C901AA
:100DC000BE010E946E34AB01EE0CFF1C65E5649F12
:100DD000C001659F900D1124E81AF90A6E2D660F67
:100DE0006E0D7E01EC18FD08FE9DD001FF9DB00D3B
:100DF00011248B2F169F70011124EF2CFF246E01FC
:100E0000CE18DF087601FE9D6001FF9DD00C1124F5
:100E10007E01E61AF108B701169F7001179FF00CCA
:100E20001124EF2CFF24CE19DF09FC9F7001FD9FD8
:100E3000F00C11247F2D43305105C1F02C3F33407D
:100E400058F441305105B1F04230510509F0A2CFBC
:100E5000EB2F8F2D7F2F9ECF4430510571F0463000
:100E6000510509F497CF7B2F8D2D94CF7D2DEB2F3E
:100E70008F2F90CF7F2FED2D8DCFEF2D7B2FF8CFA4
:100E8000282F269F020E20E0211D1124822F089575
:100E90009C0180E090E0269F020E811D369F800D10
:100EA000911D1124830F911D08959C01823091059D
:100EB00008F408959FEF213E8EE1380740F4C90100
:100EC00045E0969587954A95E1F798E0980F61E09F
:100ED000E62FE90FFF27FF1FAF0155954795842F98
:100EE000449FF001459FF00DF00D11242E173F0790
:100EF00038F49FEF940F961758F78FEF860F0895E9
:100F00004F3FE9F361E0640FF6CF40910701509144
:100F1000080125E038E0429FC001439F900D529F99
:100F2000900D1124875E994C9093080180930701DE
:100F3000890F0895982FE82F96FDE0958E2F8F70DA
:100F400096FD8F5FE695E695E695E670F0E0E85C45
:100F5000FE4F2181289F202D812D112422952F7055
:100F60008295807F282B8081820F97FD8195805804
:100F70000895FC019B01009719F4832F8078089550
:100F8000AC0197FF04C044275527481B590BB901F2
:100F9000640F751F37FD0FC0C901841B950BA5E0B9
:100FA000880F991FAA95E1F70E94823480E2861B80
:100FB000F7FD81950895CB0165E0880F991F6A952B
:100FC000E1F7BA01621B730B0E94823480E6EFCF17
:100FD0001F93CF93DF93D62FC72F182F822F86957D
:100FE000A9DF805887FD8195612F880F49DF6D2F1C
:100FF0007C2FDF91CF911F9108950F931F93CF9373
:10100000DF93162FC72FD82F022FE42FF0E0EE0F1B
:10101000FF1FE058FE4F64EE808132DF6C2F70E0DE
:10102000482F50E0445E5F4F202F30E0CA01801B04
:10103000910997FF03C0C901841B950B23E0880F1A
:10104000991F2A95E1F79B01281B390BC90137FF2E
:1010500002C080E090E06C2F13DF782F612F8D2F7E
:10106000DF91CF911F910F9108950F931F93CF930D
:10107000DF93162FD72FC82F022FE42FF0E0EE0FAB
:10108000FF1FE058FE4F64EE8081FADE6C2F70E0A7
:10109000482F50E0445E5F4F202F30E0CA01801B94
:1010A000910997FF03C0C901841B950B23E0880FAA
:1010B000991F2A95E1F79B01281B390BC90137FFBE
:1010C00002C080E090E06C2FDBDE612F7D2FDF918E
:1010D000CF911F910F9108950F931F93CF93DF939B
:1010E000162FC72FD82FBA01C9012C2F201B022F72
:1010F00040DF982F990F990F891B6C2F800FC0DE4E
:10110000782F612F8D2FDF91CF911F910F9108952F
:101110000F931F93CF93DF93162FD72FC82FBA01AA
:10112000C9012C2F201B022F24DF982F990F990F14
:10113000891B6C2F800FA4DE612F7D2FDF91CF9153
:101140001F910F910895EF920F931F93CF93DF9309
:10115000162FC72FD82FBA01C9010E190C0F09DF9E
:101160006C2F081B802F8CDE782F612F8D2FDF9145
:10117000CF911F910F91EF900895EF920F931F93CE
:10118000CF93DF93162FD72FC82FBA01C9010E199D
:101190000C0FEFDE6C2F081B802F72DE612F7D2F6E
:1011A000DF91CF911F910F91EF900895622F0895D5
:1011B000E42FF0E0EE0FFF1FE058FE4F6081621B4E
:1011C0000895E42FF0E0EE0FFF1FE05BFE4F61A9F2
:1011D000621B0895322F50E0FA01EE0FFF1FE05B13
:1011E000FE4F91A9905297FD9195440F551FFA011A
:1011F000E058FE4F2081231B330B290F311D97FD33
:101200003A95620F0895EF920F931F9310E09801A3
:10121000220F331F200F311F359527956E2D620F3A
:101220001F910F91EF9008950F93CF93DF93D72FD6
:10123000C82FB90147FD419528E330E0241B31094F
:1012400047FD3395229FA001239F500D500D11247F
:10125000669FC001679F900D900D1124840F951F0C
:1012600024DE982F990F692F680F600F7D2F8C2F28
:10127000DF91CF910F9108950F93CF93DF93D72FE5
:10128000C82FBA01C90175DE682F600F7D2F8C2F22
:10129000DF91CF910F910895EF920F93CF93DF934A
:1012A000D72FC82FBA01C9010E1963DE602F681B42
:1012B0007D2F8C2FDF91CF910F91EF9008950F9399
:1012C0001F93522F10E0F801EE0FFF1FE05BFE4F5F
:1012D000A1A9A052BB0B9D015203F001539FF00D39
:1012E0001124000F111FD801A058BE4F2C91205778
:1012F000330B4203D001439FB00D11249F012A0FED
:101300003B1F37FF02C021583F4F220F232F221FC0
:10131000330B620F1F910F9108950F931F93522F5C
:1013200010E0F801EE0FFF1FE05BFE4FA1A9A052F5
:10133000BB0B9D015203F001539FF00D1124000FD0
:10134000111FD801A058BE4F2C912057330B4203D8
:10135000D001439FB00D11249F012A0F3B1F37FF7F
:1013600002C0215C3F4F96E0359527959A95E1F7AD
:10137000620F1F910F9108950F931F93A42F10E0F8
:10138000F801EE0FFF1FE058FE4F9081905797FD38
:101390009195000F111FF801E05BFE4F01A900526B
:1013A000110B2003A001219F500D112428E330E0F0
:1013B000291B310997FD33951A2F1203F001139F52
:1013C000F00D11244E0F5F1F9A01220F331F240FBF
:1013D000351F37FF02C021583F4F220F232F221FF6
:1013E000330B620F1F910F9108951F93CF93DF93DB
:1013F000162FD72FC82F822F86959CDD805887FD0A
:1014000081956CE0880F3CDD682F610F7D2F8C2F5C
:10141000DF91CF911F9108950F931F93CF93DF9387
:101420008B01D82FC42F822F85DDEC2FF0E0EE0F3B
:10143000FF1FE058FE4F90819058890F87FD8195DE
:101440006CE0880F1DDD682F600F712F8D2FDF91ED
:10145000CF911F910F9108951F93CF93DF93162F74
:10146000D72FC82FE42FF0E0EE0FFF1FE058FE4FFC
:101470008081821B87FD819568E102DD682F610F05
:101480007D2F8C2FDF91CF911F910895CF93DF9304
:10149000D62FC72F682F842F8095F2DC6D2F7C2FDD
:1014A000DF91CF9108951F93CF93DF93162FD72FFE
:1014B000C82F60E4842F8095E3DC682F610F7D2FB7
:1014C0008C2FDF91CF911F910895EF92FF920F9390
:1014D000970195E0099F200D311D1124211591E000
:1014E000390710F02FEF30E02095382F320F08F435
:1014F0003FEF832F0F91FF90EF900895EF92FF92AF
:101500000F93E00EF11CF90137FF03C0F195E1954F
:10151000F10924E0EE0FFF1F2A95E1F7E11531E014
:10152000F30714F0EFEFF0E09A0157FF03C0319595
:101530002195310994E0220F331F9A95E1F72E1778
:101540003F070CF4F901EE0DFF1DE11591E0F907DD
:1015500010F0EFEFF0E02E2F2095382F320F08F427
:101560003FEF832F0F91FF90EF900895EF92FF923E
:101570000F93972FFA01B9019701093430F4201B1A
:101580003109211541E0340710F02FEF30E0389693
:10159000719740F0AB01485F5F4F4131510510F04A
:1015A0002FEF30E02095382F320F08F43FEF832FD4
:1015B00077FF02C06D5F7F4F75956795759567954D
:1015C0002091E503620F792F0F91FF90EF9008951E
:1015D000EF92FF920F939701201B3109211541E0F3
:1015E000340710F02FEF30E0322F3095482F430FA3
:1015F00008F44FEF842F620F0F91FF90EF90089542
:10160000EF92FF920F939701201B3109211591E072
:10161000390710F02FEF30E02095382F320F08F403
:101620003FEF832F0F91FF90EF90089590917C03EF
:10163000982B90937C030895EEC00895F7C0089509
:1016400099E0899F802D1124980F9B3208F09AE22F
:101650000895E4EEF3E0808191E089278083109281
:10166000150181E0E3CF8091E4038370811102C012
:10167000109215018091E4038C7F81608093E403D4
:1016800008958091E4038370811110921501809177
:10169000E4038C7F8093E4030895982F862F209194
:1016A000E4032370211581F0911579F0983278F4D4
:1016B0009F73990F990F2091E4032370922B9093BD
:1016C000E40310921501B2CF089591E0F2CF97E2B2
:1016D000F0CF8091E403869586958F5F883208F07D
:1016E00081E061E0DACF8091E403869586958A9562
:1016F00009F487E261E0D1CF982F822F2091E40393
:101700002370211551F09093E5036093E603453B68
:1017100008F044EB4093E70389CF0895E4EEF3E04B
:10172000818190E021E0438162810896E5CFE4EE7B
:10173000F3E0818121E0438162818850990BDCCF05
:10174000E4EEF3E0628120E1620F08F46FEF818143
:1017500021E0438190E0D0CFE4EEF3E0628120E12C
:10176000621B08F460E0818121E0438190E0C4CFF6
:10177000E4EEF3E0438120E1420F08F44FEF818172
:1017800021E0628190E0B8CFE4EEF3E0438120E114
:10179000421B08F440E0818121E0628190E0ACCFFF
:1017A000E4EEF3E0248130E1230F08F42FEF2483EB
:1017B00081E03CCFE4EEF3E0248130E1231B08F428
:1017C00020E0248381E032CF81152CE7920741F499
:1017D0002091F4033091F503232B11F480E090E085
:1017E0000895EFE9F4E080E090E061E379E244E518
:1017F00059E226EC39E27783668351874087338745
:10180000228797878687019670968530910599F78C
:101810000895239A0895FC01EE0FFF1FE80FF91FAA
:10182000E954FD4F6183408322830895FF920F9313
:101830001F93CF93DF93182F062FF42EC0E0D0E034
:101840002F2D402F612FCE01E6DF2196CA32D10520
:10185000B9F7CDB7DEB7E5E00C94E7341092280570
:1018600010922705ECEFF4E08581811102C014820B
:101870001682379685E0EF31F807B1F70895AC018D
:1018800030912A0560912905232F621301C0089524
:10189000822F90E0FC01EE0FFF1FE15EFA4F0190F6
:1018A000F081E02DE417F50791F467E0649FF00103
:1018B000659FF00D1124E450FB4F41E04483231356
:1018C000E6CF01968370992780932A0508950196A3
:1018D000282F2370DACF282F35EB2303C0011124E2
:1018E00097FF04C080589109892F089580589F4F11
:1018F000FBCF80918E0480FD14C081FD14C082FD59
:1019000016C080918D04811581F08E3180F420E520
:10191000829FC00111246EE170E00E948234862F04
:10192000089584E1089588E2089588E0089580E5A7
:10193000089580918E0480FD17C081FD17C082FD3F
:1019400019C080918C04811599F0883298F428E0B0
:10195000829FC001112468E270E00E948234611508
:10196000710551F0862F089562E0FCCF64E0FACF54
:1019700061E0F8CF68E0F6CF81E00895FA01309792
:1019800009F009950895E0911D04F0911E04309727
:1019900039F00190F081E02D309711F0099508950C
:1019A00080E00895A3E0B0E0E8EDFCE00C94CE34D4
:1019B0009C018091B4029091B50282179307B1F017
:1019C0003093B5022093B402E0911D04F0911E04FF
:1019D000309761F00084F185E02D309739F083E095
:1019E00089833B832A83CE01019609952396E2E001
:1019F0000C94EA34A3E0B0E0E0E0FDE00C94CE34D7
:101A00009C018091B2029091B30282179307B1F0CA
:101A10003093B3022093B202E0911D04F0911E04B2
:101A2000309761F00084F185E02D309739F084E043
:101A300089833B832A83CE01019609952396E2E0B0
:101A40000C94EA3490911A01913021F49091980508
:101A500097FD0CC0E2E7F2E09191891302C0DF012B
:101A60001E9252E0E837F507B9F70895E82FE6959A
:101A7000E695E695803FC8F7F0E0E858FD4F87709F
:101A800021E030E0A90102C0440F551F8A95E2F71A
:101A9000CA018095928189238283089580911901DA
:101AA00008952FB7F8948091AE029091AF02A09163
:101AB000B002B091B1022FBF0895CF93DF93C091D0
:101AC000F4048091F604C82B8091F304811501F190
:101AD000E8DF2091FA043091FB04821B930B8838D5
:101AE000934110F00E94A404D091F30480911A0154
:101AF000813021F48091980587FD0EC086E022E7B1
:101B000032E090E0815060F491110E94A404CD2B4A
:101B10008C2FDF91CF9108958EE12AE732E0F1CF4B
:101B2000F90141919F01411569F39F5FEBCF962F1A
:101B30002091990522FF0FC0682F660F660F660F70
:101B4000692B6093F7040E94D603ABDF9093F904EE
:101B50008093F80408950C94D6039091F304292FF0
:101B60002823211559F0809589238093F30481154A
:101B700031F097DF8093FA049093FB04089580E09E
:101B800090E0F8CF8EDF2091910430919204232BC6
:101B9000211521F08093DD039093DE0320919304BF
:101BA00030919404232B211521F08093DB03909333
:101BB000DC03E0911D04F0911E04309759F006807B
:101BC000F781E02D309731F082E080938F048FE829
:101BD00094E009950895611509F441C0E3E3E80F25
:101BE000E33148F4F0E0E056FA4C0C94B13481DE75
:101BF000819580939204C6CF7CDEFBCF7ADE8195FF
:101C000080939104F8CF75DEFBCF93DE809393042D
:101C1000F2CF8FDE8195FACF8CDE8195809394048C
:101C2000EACF87DEFBCF815D990B21E030E001C078
:101C3000220F8A95EAF780919004822B809390047A
:101C4000DACF80918E04816080938E04D4CF80910E
:101C50008E048260F9CF80918E048460F5CF40912C
:101C600091048D3C59F48091920487FF0DC010922D
:101C70009204411559F410928D0408C08E3C81F4F1
:101C80008091920418169CF3411581F08091930481
:101C900090919404892B8111AECF10928C04ABCF1C
:101CA0008F3C41F447FFF0CF109291048091920451
:101CB0008115E0CF803D19F41416B4F3E5CF90916F
:101CC0009304893D29F41916FCF610929304DCCF95
:101CD0008A3D19F497FFD8CFF8CF909194048B3DAB
:101CE00029F497FFD1CF10929404CECF8C3D19F4F4
:101CF0001916CCF3C9CF9FE2980F983090F4815D0C
:101D0000990B21E030E0B90102C0660F771F8A9578
:101D1000E2F7CB0180959091900489238093900401
:101D2000B3CF8D3D31F480918E048E7F80938E04ED
:101D3000ABCF8E3D21F480918E048D7FF7CF8F3D08
:101D400009F0A2CF80918E048B7FF0CF2FB7F8944B
:101D50006091AE027091AF028091B0029091B10299
:101D60002FBF0895FC019B018091A4029091A502D0
:101D70008617970740F0672B29F48091E8008E774B
:101D80008093E800C90140E0009741F4411106C08A
:101D90008091E80082FF2FC080E008952091F60333
:101DA0002115A9F12530A9F12091E80023FD2DC0CE
:101DB0002091E80022FDECCF2091E80020FFE4CF45
:101DC0003091F3002091F200009719F0283031058E
:101DD00058F041E02830310509F040E02091E8005A
:101DE0002E772093E800D0CF41914093F1000197E6
:101DF0002F5F3F4FE9CF8091F603811541F0853089
:101E000041F08091E80083FFC3CF81E0089582E034
:101E1000089583E0089580919E0287FF13C080910A
:101E2000E80082FF06C08091E8008B778093E8008D
:101E300008958091F6038111F2CF08958091F60301
:101E40008115D9F38091E80080FFF8CF8091E800F8
:101E50008E77ECCF2091E4003091E50095E6A90162
:101E60002091EC00822F817020FF06C08091E80055
:101E700080FF06C080E008952091E80022FD1AC08E
:101E80008091F603811589F0853089F08091EB000F
:101E900085FD0FC02091E4003091E5004217530703
:101EA000F9F29A95E1F684E0089582E0089583E0DE
:101EB000089581E00895E8EDF0E080818E7F8083D1
:101EC0001092E2001092DA001092E100A0EEB0E071
:101ED0008C9181608C9380818F77808319BCA7ED72
:101EE000B0E08C918E7F8C9380818F7E8083109266
:101EF0009D020895E0911D04F0911E04309739F081
:101F00000284F385E02D309711F060E20995089581
:101F1000AF92BF92DF92EF92FF920F931F93CF93F6
:101F2000DF935C01809104018BDBC82F192F609136
:101F3000E803669580917003909171030E944807B1
:101F4000D82ED0E0CE01880F991F9C01205B3E4F18
:101F500079011C1709F070F481E01A3208F080E072
:101F6000DF91CF911F910F91FF90EF90DF90BF9085
:101F7000AF900895FE01EC52FE4F808190910501D3
:101F800089238115B1F0F70121A92052330B40A913
:101F90004057550B6091E5037091E6038091E7038C
:101FA0000D2DF50109950E94B906472F282FCE0166
:101FB00043DBF2E0EF0EF11C2196CBCFA0E0B0E0C6
:101FC000E4EEFFE00C94C2343C018091040138DB64
:101FD000C82F192F6091E803669580917003909146
:101FE00071030E944807F82ED0E0CE01880F991F98
:101FF0009C01205B3E4F69011C1709F048F481E009
:102000001A3208F080E0CDB7DEB7EEE00C94DE3493
:10201000FE01EC52FE4F80819091050189238115CC
:1020200069F1F60180A9282F2057330B590181A9A6
:10203000E82FE052FF0B4F01AA9C9001AB9C300DA2
:10204000300D1124EE9FC001EF9F900D900D1124D3
:10205000820F931F0E945507082F6091E50370912E
:10206000E6038091E703EF2C9401A501F3010995A4
:102070000E94B906472F282FCE01DEDAF2E0CF0EFC
:10208000D11C2196B9CFA4E0B0E0E9E4F0E10C94D2
:10209000C8346C0180910401D3DA8B83F92E6091EE
:1020A000E8036695669580917003909171030E9494
:1020B0004807182F80E4810F0E949A07805889836F
:1020C000812F0E949A0780588A839B81892F90E0F4
:1020D0009C838B839B819F1548F081E0EAE2FE168A
:1020E00008F080E02496E8E00C94E434EB81FC8175
:1020F000EC52FE4F8081909105018923811599F062
:102100006091E5037091E6038091E703E12E0B8176
:102110002A814981F60109950E94B906472F282F87
:102120008B819C8189DA8B819C810196D1CFCF9262
:10213000DF92FF920F931F93CF93DF93C82FD0E0CE
:10214000FE01EC52FE4F808190910501892381159B
:1021500071F1F090E6030091E7031091E503C12EC1
:10216000D12C0E948507482FC6018C549F4F68E6EA
:1021700071E00E9482348C199D0997FD03969C01A1
:102180003595279535952795842F90E0AC01440F20
:10219000551F840F951F612F299F600D11247F2DDE
:1021A000802F0E94B906472F282FCE0145DADF91F4
:1021B000CF911F910F91FF90DF90CF9008951F93C3
:1021C000CF93DF93C82FD0E0FE01EC52FE4F808109
:1021D0009091050189238115A1F00E948507182F90
:1021E0000E94850720E8829FC00111247FE7790FB4
:1021F000612F8091E7030E94B906472F282FCE0157
:102200001BDADF91CF911F910895EF92FF920F9308
:102210001F93CF93DF937C018091040111DAC82FC3
:10222000192F6091E8036695669521E0620F08F426
:102230006FEF80917003909171030E944807082FFF
:10224000D0E0C11748F081E01A3208F080E0CDB745
:10225000DEB7E6E00C94E634FE01EC52FE4F8081DE
:10226000909105018923811581F06091E5037091BA
:10227000E6038091E703202F4C2FF70109950E9478
:10228000B906472F282FCE01D7D92196DACFA0E063
:10229000B0E0EDE4F1E10C94C7348C0180910401CD
:1022A000CFD9C82FD92E2091E80331E0230F08F4AD
:1022B0002FEF30E040E050E06FEF7FEF80E090E004
:1022C0000E9495347901D0E0C22EBF2C2C2FCD1561
:1022D00050F081E0FAE2DF1608F080E0CDB7DEB71B
:1022E000E9E00C94E334FE01EC52FE4F80819091C2
:1022F00005018923811509F140917D034150042E88
:10230000000C550B47FF1BC08C2D9B2D6091E803E3
:1023100021E0620F08F46FEF0E944807AC01609162
:10232000E5037091E6038091E703F80109950E94A7
:10233000B906472F282FCE017FD92196C7CFFA01A2
:10234000E358FC4F818982130AC0FA01EE0FFF1F88
:10235000E358FC4F818D928D8E159F05B8F2415048
:102360005109D0CFA8E0B0E0E8EBF1E10C94BE3425
:10237000382E6A837B838091040162D9192F2091C2
:102380007D032E83E82FF0E0F887EF83CF01880FDD
:10239000991F9C01205B3E4F6901432C512C3FEF5C
:1023A000431A530A8F81811740F081E01A3208F0F6
:1023B00080E02896E2E10C94DA34EF81F885EC5263
:1023C000FE4F80819091050189238115E9F080916C
:1023D000E5038C839091E6039D83F201E358FC4F63
:1023E0003F01232C1982FE812F16C0F06091E70374
:1023F00089810E9440076C817D810E94B906472F28
:10240000282F8F81988518D92F8138852F5F3F4FCE
:1024100038872F8332E0C30ED11CC4CFF3018191E2
:102420003F01F601A0A8A81ABB0881A8F301878183
:10243000881A9908AA9C9001AB9C300D300D11248C
:10244000889CC001899C900D900D1124820F931FD0
:102450000E945507082F6091E80321E0620F08F4FD
:102460006FEFF301EE0FFF1FED57F340858996895B
:102470000E9448077C019401A5016C817D818981BE
:10248000EA81FB8109956C837D8389832394ABCF9B
:10249000A0E0B0E0EEE4F2E10C94C634C82F8091E5
:1024A00017018C1321C09091E403937020911601C1
:1024B00030E081E09217130609F480E08093060172
:1024C0008091E90390910501981731F080930501FF
:1024D00040E060E080E0B2D8C83280F4EC2FF0E059
:1024E000ED54FA4C0C94B13481E0E8CF80910601B0
:1024F000811521F040E060E080E0A0D880E0D8C005
:10250000809104019DD8082FD92F6091E503709127
:10251000E6038091E7030E94B906F62EE72ED82E37
:1025200010E0D01709F018F481E0DA3236C0F80173
:10253000EC52FE4F8081909105018923811529F08D
:102540002D2D4E2D6F2DC80177D80F5F1F4FE9CF6E
:102550008091040175D8082FD92ED091E503F09011
:10256000E6031091E7036D2F7F2D812F0E94B9069E
:10257000C62EB72EA82E8091E8036D2F680F7F2DF1
:10258000812F0E94B906D62FF72EE82E10E0D01624
:1025900009F030F481E02AE2D21608F489C0AECF07
:1025A000F801EC52FE4F808130910501382331153E
:1025B00051F02E2D4F2D6D2F80FD03C02A2D4B2D58
:1025C0006C2DC80139D80F5F1F4FE1CF80910401F6
:1025D00037D8082FD92FE090E603D090E703609119
:1025E000E80380E40E944007F82E10E0D01709F0BD
:1025F00008F49ACFF801EC52FE4F808190910501CA
:1026000089238115A9F0F801EE0FFF1FE05BFE4F53
:1026100081A982958F706091E5038F9D600D1124D3
:102620007E2D8D2D0E94B906472F282FC80104D872
:102630000F5F1F4FDBCF8091040102D8082FD92FE5
:10264000E090E603D090E7036091E80380E40E9405
:102650004007F82E10E0D01709F008F465CFF80114
:10266000EC52FE4F80819091050189238115D1F0B4
:10267000F801EE0FFF1FE05BFE4F20A92F9D900198
:10268000112495E0359527959A95E1F76091E5033A
:10269000620F7E2D8D2D0E94B906472F282FC8016D
:1026A0000E941C0B0F5F1F4FD6CF88EE97E0ADDD69
:1026B000909104019F5F9093040181110CC082E00E
:1026C0008093150180910601811105C0C11103C0DD
:1026D00083E080931501CDB7DEB7EAE00C94E234D5
:1026E0008DEF97E0E4CF85E398E0E1CF8CE698E0CA
:1026F0000FDCDECF88E898E0FBCF83EA98E05EDC71
:10270000D7CF8DEB98E0FBCF86ED98E0D0CF88ED6A
:1027100098E0CDCF81EE98E0CACF8AEE98E0C7CF9F
:1027200083E099E0ECCF84E199E0E2CF8CE399E09B
:10273000DFCF8CE499E0E3CF8FE599E0A4DCB8CF5C
:102740008DE899E0FBCF8CEB99E0F8CFD0910401B4
:10275000D1111FC06091E80320E1620F08F46FEF10
:1027600080917003909171030E9448076AE070E0C5
:102770000E946E34892B69F40E9485073AE2839F98
:10278000C0011124892F880F880B9093000180933A
:1027900001018D2F0E94200B282F192F082F8091C7
:1027A0000601811115C080910001909101018217ED
:1027B000910580F08117910568F4B9DC8BE290E017
:1027C000909301018093000105C0802FB0DC0F5F62
:1027D0000117D8F381E01A32E0CED0910401D11173
:1027E0001FC06091E80320E1620F08F46FEF809151
:1027F0007003909171030E94480765E070E00E94A9
:102800006E34892B69F40E9485072AE2829FC001F9
:102810001124892F880F880B909302018093030164
:102820008D2F0E94200B282F192F082F8091060131
:10283000811115C0809102019091030182179105C9
:1028400048F28117910530F6BADC8BE290E0909364
:10285000030180930201BECF802FB1DC0F5F01170F
:10286000D8F3B8CF85EF99E022CF8CE09AE01FCF64
:102870008CE29AE01CCF86E49AE009DD19CF83E56B
:102880009AE0FBCF80917D0321E0382F321B08F4C2
:1028900030E0832F65E67AE065DD0ACF65E67AE011
:1028A00080E0FACF80917D0321E0382F321B08F4BD
:1028B00030E0832F6EE77AE0EFCF6EE77AE0F0CF7B
:1028C00080917D0321E0382F321B08F430E0832F04
:1028D00066EB7AE0E1CF66EB7AE0E2CF80917D03B0
:1028E00021E0382F321B08F430E0832F68EE7AE0C5
:1028F000D3CF68EE7AE0D4CF80917D0321E0382FEA
:10290000321B08F430E0832F60E07BE0C5CF60E04D
:102910007BE0C6CF982F9093E900891771F07091F2
:10292000EC002091ED005091F00021FD09C09F5F67
:10293000973089F78093E9000895762F242F50E08F
:102940003091EB003E7F3093EB003091ED003D7F06
:102950003093ED003091EB0031603093EB007093D9
:10296000EC002093ED005093F0002091EE0027FD45
:10297000DECF0895A0E0B0E0E0ECF4E10C94C834C0
:10298000C8EDD0E088818F7E8883E7EDF0E080811C
:102990008160808384E082BF81E080939D02888192
:1029A0008E7F888302EE10E0F80110821092DA0028
:1029B00081EEC82ED12CF601108288818F77888312
:1029C00088818068888388818F7D888319BC109274
:1029D000F60310929C021092A80310929B0290EEB4
:1029E000E92EF12CF70180818B7F808388818160C3
:1029F000888342E060E080E08DDFF60180818E7F99
:102A00008083F801808181608083808188608083F9
:102A1000F70180818E7F8083888180618883CDB734
:102A2000DEB7E8E00C94E434E091280490912704A8
:102A300029E0E91302C080E00895AE2FB0E02E9F98
:102A4000F0011124E75DFB4F3181361306C0308160
:102A5000381303C03581341304C0FD013196E7708B
:102A6000E8CF81E0089535B1377F25B128604FB7B1
:102A7000F89487EB92E0FC010196508168E025B95B
:102A8000000000C057FF35B9550F000000C000C05E
:102A900000C035B900C06A9591F753E085339507BA
:102AA00051F74FBF8FE594E00197F1F700C00000A8
:102AB000089581E08093E00080E28093D800109236
:102AC000C9008FE19EE40197F1F700C0000087E0A4
:102AD00090EBDC0180939A0590939B05A0939C0555
:102AE000B0939D0588E19CE00FB6F894A89580937B
:102AF00060000FBE90936000FFCF0F931F93CF93A2
:102B0000DF938B01EA019091F603943051F58093A5
:102B1000E9008FEF9091E80095FD06C095ED9A953C
:102B2000F1F700008A95B1F78091E80085FF19C0A0
:102B300091D9811111C08091E80085FD06C0809176
:102B4000E8008E778093E800F3CFF80181918F0140
:102B50008093F100219779F78091E8008E77809338
:102B6000E800DF91CF911F910F910895792F603286
:102B700029F440E250E0682F82E0BFCF0895CF9360
:102B8000DF93D82FC92F48E050E0682F792F81E0DC
:102B9000B4DF88E0ED2FFC2FA6EAB2E001900D92A1
:102BA0008A95E1F7DF91CF910895BC0140E250E0B2
:102BB00084E0A3CFBC0146E050E084E09ECFBC019E
:102BC00043E050E084E099CF9091990592FB222751
:102BD00020F9281779F080FB92F99093990560917C
:102BE00098057091990584E090E00E94833582E019
:102BF0000C94810408951F93CF93DF93962F122F87
:102C0000632F282F292B2430C8F44C30B8F4C42F5C
:102C1000D0E0CC0FDD1F28E1929FC00DD11D112403
:102C200090E6899FC00DD11D1124CE0189960E9486
:102C30006935612FCE018A960E946935DF91CF9167
:102C40001F91089580911A01813069F5809198054E
:102C500087FF29C00E945D0D8093790240E250E019
:102C60006DEF73E088E792E00E942035892BD1F068
:102C700080E2E8E7F2E0ADEFB3E001900D928A95D3
:102C8000E1F7E0911D04F0911E04309759F00480A3
:102C9000F581E02D309731F086E08093780288E767
:102CA00092E0099508950E945D0D8093700248E0BE
:102CB00050E06FE174E080E792E00E942035892BBC
:102CC00089F388E0E0E7F2E0AFE1B4E001900D9233
:102CD0008A95E1F7E0911D04F0911E04309711F3FD
:102CE0000280F381E02D3097E9F280E792E0D9CFBE
:102CF000CF93C82F811509F464C08CEF8C0F813AF3
:102D000008F061C080911A01813031F1E2E7F2E010
:102D100088E792E02191C217C9F18E179F07D1F77A
:102D200080911A018130B9F1A2E7B2E0EFEF80E0C3
:102D30009D91C91709F444C0EF3F19F4911101C0E6
:102D4000E82F8F5F8630A1F7EF3FD1F10E2E000CF8
:102D5000FF0BE059FD4F33C08091980587FFD6CF18
:102D6000EC2FE695E695E695F0E0E858FD4F828178
:102D700090E04C2F477021E030E002C0220F331F5B
:102D80004A95E2F782239323892B29F08C2F0E9406
:102D9000220D58DFC5CF8091980587FFC5CFEC2F56
:102DA000E695E695E695F0E0E858FD4FC77081E0BE
:102DB00090E001C0880FCA95EAF7C281C82BC28390
:102DC00041DFCF91089580E28C0F883068F4C7709E
:102DD00081E090E001C0880FCA95EAF7C091F40441
:102DE000C82BC093F404ECCF8BE58C0F833038F400
:102DF0002C2F2452330BC9010E94D20CE2CFE8E5FC
:102E0000EC0FEB3150F4F0E0EE0FFF1FE85CFD4FEC
:102E1000808191810E94FA0CD4CF83E38C0F83319F
:102E200080F661E08C2F0E94EB0DCBCF811561F114
:102E30009CEF980F913A18F40E94220D03CF90E274
:102E4000980F983050F4877091E001C0990F8A95DF
:102E5000EAF7892F0E949C04F1CF9BE5980F9330ED
:102E600020F480E090E00C94D20C98E5980F9B3110
:102E700020F480E090E00C94FA0C93E3980F9331E7
:102E800018F460E00C94EB0D08951F93CF93DF933B
:102E9000182FEB012DDF209731F4812FC7DFDF9151
:102EA000CF911F9108958FE99FE00197F1F700C03E
:102EB00000002197F0CF811531F09091F404892B17
:102EC0008093F404BFCE0895811519F00E949C04EC
:102ED000B9CE0895811531F09091F604892B809335
:102EE000F604B0CE0895811539F080959091F604DE
:102EF00089238093F604A6CE08951092F40480915D
:102F00001A01813029F58091980587FF21C0EAE7F1
:102F1000F2E08EE1DF011D928A95E9F780E090E012
:102F20000E94D20C80E090E00E94FA0C1092F6040D
:102F300089DE86E0EFE8F4E0DF011D928A95E9F78B
:102F400010928D0410928C0410928E040C94C20D79
:102F5000E2E7F2E086E0DECFD0DF2FEF84E39CE013
:102F6000215080409040E1F700C0000088E19CE0E3
:102F70000FB6F894A895809360000FBE9093600000
:102F8000FFCFAAE2B0E0E7ECF7E10C94CD348EE994
:102F900092E0FC0101962091F100208322E0863A24
:102FA0009207B9F780919F02893009F459C0C8F49B
:102FB000823009F4B6C0833009F485C0813089F1CC
:102FC0008091E80083FFEAC080919E0290919F0269
:102FD0009A3008F0E3C0E92FF0E0E552FA4C0C9487
:102FE000B1348A3009F48CC08B3051F780919E0245
:102FF000813231F78091A2029091A302892B01F7CF
:103000008091E800877F8093E8000E940B0F81E0A9
:103010009091A002911101C080E080931A016DDFB0
:10302000CFCF80919E02813A59F68091E800877F48
:103030008093E8008091A2029091A302892B61F015
:1030400060E080E090E070E00E94B20E8091E800C5
:103050008B778093E800B4CF68E086EA92E0F3CF04
:1030600080919E02813209F0ABCF8091A2029091B3
:10307000A3028D7F892B09F0A3CF8091E800877F81
:103080008093E8008091E80082FF18C09091F300DF
:103090008091F200029731F48091F100813011F0BB
:1030A000863021F48091F100809319018091E8002D
:1030B0008B778093E8000E940B0F82CF8091F603FC
:1030C0008111E0CF7DCF80919E02813A09F078CFC7
:1030D0008091A2029091A302892B09F071CF809177
:1030E000E800877F8093E8008091E80080FFFCCFB4
:1030F00080911A018093F1008091E8008E77D9CFFA
:1031000080919E02813209F05BCF8091E800877F39
:103110008093E8000E940B0F8091A1028093180118
:103120004FCF80919E02813A09F04ACF8091E8000A
:10313000877F8093E8008091E80080FFFCCF80913A
:103140001801D8CF803889F0823841F58091A202E9
:103150008F70873018F58093E9008091EB0085FB34
:10316000882780F91092E90006C08091A803880F93
:1031700090919B02892B9091E800977F9093E800B3
:103180008093F1001092F1008091E8008E7723C0C7
:10319000811116C08091A002813011F18091E80068
:1031A00083FF0AC08091E800877F8093E8008091C8
:1031B000EB0080628093EB00AA96E3E00C94E93484
:1031C000823061F78091A002811589F01092E900A8
:1031D0008091E800877F8093E8000E940B0FDECF8C
:1031E00081E0933009F080E08093A803EFCF8091D5
:1031F000A2028F702FEF280F263080F68093E9000F
:103200002091EB0020FFE2CF933031F48091EB006E
:1032100080628093EB00DACF9091EB009061909305
:10322000EB0021E030E0A90102C0440F551F8A9550
:10323000E2F74093EA001092EA008091EB00886088
:10324000E8CF8111ABCF1091A0021F778091E300EE
:103250008078812B8093E3008091E800877F8093C2
:10326000E8000E940B0F8091E80080FFFCCF809166
:10327000E30080688093E30083E0111101C082E0E5
:103280008093F6038BCF8058823008F087CF8091EF
:10329000A0029091A1028C3D53E0950799F583E03F
:1032A0008A838AE289834FB7F894DE01139620E07F
:1032B0003EE051E2E32FF0E050935700849120FF6D
:1032C00003C082958F703F5F8F708A30C8F0895C31
:1032D00090E08D939D932F5F243161F74FBF8091D4
:1032E000E800877F8093E8006AE270E0CE010196F3
:1032F0000E94B20E8091E8008B778093E8004ECF59
:10330000805DE6CF292F33272330310509F44EC0E5
:1033100078F52130310509F488C08BE590E0E8E7C5
:10332000F2E02230310509F039CF2091E800277F03
:103330002093E8002091A4023091A5028217930700
:1033400008F49C0140E02115310509F073C04111DA
:1033500071C08091E80082FDCDCF8091F603811588
:1033600049F2853039F28091E80083FFF2CFC2CF75
:103370008091A2029091A3022132310509F446C046
:103380002232310509F00ACF8330910508F006CFCB
:10339000FC01EE0FFF1FE45DFE4F0190F081E02D78
:1033A000875D9E4FDC018C9190E010C09C0133271B
:1033B000823021F12330310568F4232BB9F4EDE29A
:1033C000F3E0E4918E2F90E0EDE2F3E0009709F452
:1033D000E5CEABCF2330310509F0E0CEE5EEF2E0EB
:1033E000E4918E2F90E0E5EEF2E0F0CFEDE1F3E036
:1033F000E4918E2F90E0EDE1F3E0E8CFE3E0F3E03D
:10340000E4918E2F90E0E3E0F3E0E0CF833091058C
:1034100008F0C4CEFC01EE0FFF1FEE5CFE4F0190E2
:10342000F081E02D89E090E080CF82E190E0E3ED53
:10343000F2E07BCF8091F603811509F45BCF8530F4
:1034400009F458CF8091E80083FD54CF8091E800C3
:1034500082FD7FCF8091E80080FF75CF9091F300CF
:103460008091F2002115310519F08830910550F056
:1034700041E0089709F040E08091E8008E77809362
:10348000E80061CF44914093F10031962150310919
:103490000196E8CF803809F081CE8091E800877FDF
:1034A0008093E80080919C028093F1006DCE8111A1
:1034B00075CE1091A002123008F070CE8091E80015
:1034C000877F8093E80010939C020E940B0F1115D8
:1034D000D9F084E08093F60342E061EC81E01ADAEF
:1034E00042E261EC84E016DA42E261EC82E012DA58
:1034F00042E260EC83E00EDA8091F603843051F40E
:1035000082E080931B014ACE8091E30087FDE1CFEA
:1035100081E0E0CF81E0F5CFCF93DF93EC014A85E6
:103520005B856E857F850E94BE0C9B819095809106
:10353000F60489238093F6048C810E949C0482DB2C
:1035400086E0FE0111928A95E9F7DF91CF91089507
:10355000CF93DF93EC018D8181FD16C082608D8356
:103560008091F6049B81892B8093F6048091F4046A
:103570009C81892B8093F40465DB488559856E8591
:103580007F85CE010E94BE0C1092F0041092EF04D1
:103590008D8180FD02C0CE01BFDFDF91CF91089504
:1035A0000F931F93CF93DF93982F962B943020F592
:1035B0004C3010F5C42FD0E0CC0FDD1F28E1629F06
:1035C000C00DD11D112430E6839FC00DD11D1124E3
:1035D000CE0189960E944D35082F10E0102F00274C
:1035E000CE018A960E944D359801282BC901DF91A2
:1035F000CF911F910F91089580E090E0F8CF462F72
:10360000672F2091F9033091FA03232B81F4703F47
:1036100039F4403F61F48091F7039091F8030895E5
:10362000982F972B943018F44C3008F4B9CF80E0E1
:1036300090E00895A0E0B0E0E0E2FBE10C94C93432
:103640007C010091970580919605082BC3E0D0E09E
:1036500010E0C8010C2E02C0959587950A94E2F7F8
:1036600080FD09C02197A8F7D12C8D2DCDB7DEB7ED
:10367000E7E00C94E534DC2EB7018C2FC0DF0E940C
:10368000A205019779F3F1CF0F931F93CF93FC011C
:1036900087819085009789F485810081118181154A
:1036A00081F0611571F0C801C5DFC82F682FC8010E
:1036B0000E94EE03B8018C2FA2DFCF911F910F91D2
:1036C0000895C8010E942404C82FF4CFCF93DF933C
:1036D000D82FC92FAFDF6D2F7C2F91DF0E94A2055D
:1036E000DF91CF910895FC0184818115B1F087812C
:1036F00090850097A1F00E94A205282F92959F70B7
:103700009630B9F080F4925F9F70923030F4203F91
:10371000D1F058F481E0283E58F080E0089580818F
:103720009181D4DFEACF9A5FEFCF81E0243FA9F700
:10373000089591E0813F09F090E081E0283E08F093
:1037400080E0892B089581E00895382F292FCB013F
:10375000A32FB22F833F21E09207A105B10520F4EA
:10376000835F9D4F0C944D3580E0089585E290E095
:103770000E944D35803D89F486E290E00E944D35EF
:10378000893559F487E290E00E944D3591E0893205
:1037900009F090E0892F8170089580E0FCCFAAE0C5
:1037A000B0E0E5EDFBE10C94C334C090F403D0909D
:1037B000F50381E090E09093F5038093F403812C6E
:1037C000912CE12C5401F12C14C0F8012591359174
:1037D000472D6F2D8E2D0FDA0E5F1F4F73948CE0E7
:1037E0007812F3CF9CE0A90EB11CF394E4E0FE162E
:1037F00039F08501000F111F0F5C1C4F712CE5CFB4
:10380000E394F0E38F0E911C84E0E812DBCF1A8280
:1038100019821C821B821E821D8218861F8288ECE0
:1038200090E09A87898709EA11E0FE0131967F01CD
:103830004AE050E0B801C7010E948735065F1F4F7C
:1038400057010B3DF1E01F0799F78AE0F70111924C
:103850008A95E9F74AE050E0B801C5010E94873532
:10386000065F1F4F0D30F2E01F07A1F7D092F5035E
:10387000C092F4032A96EDE00C94DF34AAE0B0E0A5
:10388000E4E4FCE10C94C834E5E3F3E082E3DF0117
:103890001D928A95E9F7ECEFF4E083E2DF011D92D7
:1038A0008A95E9F785E3C82E83E0D82E7F010BEDDA
:1038B00011E0F701D182C0824AE050E0B801CE01A8
:1038C00001960E943D3588E0FE013196D6010190B7
:1038D0000D928A95E1F789859A85D70113969C9375
:1038E0008E931297BAE0CB0ED11CE7E0EE0EF11CDE
:1038F000065F1F4F0D30F2E01F07D9F62A96E8E069
:103900000C94E434282FCB01253070F44AE0249F36
:1039100090011124B90167557E4F4AE050E00E94A2
:103920003D3580E090E008958FEF9FEF0895AAE085
:10393000B0E0EDE9FCE10C94CE349C019755811583
:10394000914068F4BE016F5F7F4F822FDBDF892BD0
:1039500031F489859A852A96E2E00C94EA3488EC61
:1039600090E0F9CFA8E0B0E0E8EBFCE10C94C234C1
:10397000FE01319688E0DF011D928A95E9F790E417
:10398000A92E91E0B92E8F013F01EE24E394F12C92
:1039900030E5C32E31E0D32EF50181915F018F3FD9
:1039A00009F444C0F894E82FE295EF70F0E021A10B
:1039B0008F70A70102C0440F551F8A95E2F7CA0114
:1039C000922F982B91A392A18095892382A378941A
:1039D00000C0E4E4F1E021E030E0812C912C419141
:1039E0004F3F79F0A42FA295AF70A05EB0E08C910C
:1039F00090E04F7002C0959587954A95E2F780FF59
:103A00003BC080E090E0882A992A220F331FCE160F
:103A1000DF0629F7F50182918F3F11F00E94A00681
:103A200050EA5A95F1F7D8018D929C920E5F1F4F84
:103A3000B4E4AB16B1E0BB0609F0AECF48E050E00D
:103A4000B30184E793E00E942035892BB9F088E028
:103A5000F301A4E7B3E001900D928A95E1F781E0CC
:103A600080939A020E94510D90939902809398023C
:103A70002896EEE00C94DE34C901C5CF80919A02FD
:103A80008115B1F300919802109199020E94510D95
:103A9000801B910B059760F348E050E064E773E00A
:103AA0008CEE93E00E942035892B49F088E0E4E712
:103AB000F3E0ACEEB3E001900D928A95E1F710923D
:103AC0009A02D6CFA0E0B0E0E8E6FDE10C94C7345E
:103AD000EC018881811509F1813009F045C08981A7
:103AE000813051F48A81239660E570E0893311F0CA
:103AF00060E070E0CAD9EDCF823021F48A8123964C
:103B0000F7D8E7CF833021F48A8123968FD9E1CF8C
:103B1000843041F022968111DCCFCDB7DEB7E9E0E9
:103B20000C94E3348A81239620E030E09AE0682FF9
:103B30006053770BAB016A30710560F021153105D8
:103B400051F3EFE9FFE03197F1F700C00000215099
:103B50003109F4CF929FB001939F700D11249A0107
:103B6000260F371F8991E3CFE82FF0E0E850FE4F92
:103B7000B490282F26952695269530E0F901E85136
:103B8000FE4FE4908770F12C082E02C0F594E79464
:103B90000A94E2F7E0FAEE24FF24E0F8F901E85293
:103BA000FE4FC490D12C082E02C0D594C7940A941D
:103BB000E2F7C0FACC24DD24C0F8F901E853FE4F47
:103BC000049110E002C0159507958A95E2F70170FF
:103BD0001127E114F10411F081EE8AD8C114D10447
:103BE00011F086EE85D860E070E08B2D4ED9C114BF
:103BF000D10411F086EE1AD9E114F10411F081EE2E
:103C000015D90115110521F060E070E08CE23DD975
:103C100021965FCFA6E0B0E0E0E1FEE10C94BE3477
:103C20008D839E83AD81BE8114968C9114978115EE
:103C300009F4E3C161E0CD0127DD8C01ED81FE8156
:103C40008581811519F18091EF049091F00400971E
:103C5000E9F008171907D1F0FC01FF27853008F0BB
:103C60006FC074E0EE0FFF1F7A95E1F7E156FB4F4E
:103C700085818460858311830083CF0169DC109284
:103C8000F60461E08D819E81FFDC8C01AD81BE81F7
:103C900015968C91811509F4D8C0C80197578038C2
:103CA000910508F0EEC0053008F095C162EF71E0B3
:103CB00080E090E04ADD81118EC1C12CD12C7601CB
:103CC000011141C064E0362E8E010F5F1F4FD801F5
:103CD000E32D1D92EA95E9F746015701FFEF8F1A90
:103CE0009F0AAF0ABF0AC701B6012FDD898381157C
:103CF00009F471C1813009F0A5C02601370122E025
:103D0000420E511C611C711CC501B4011EDD282E20
:103D10008A83811509F45FC18FEF820D833038F5F6
:103D2000C301B20112DD8B83811511F0C801CADE17
:103D30004601570143E0840E911CA11CB11C45C0F3
:103D4000E0E0F0E095CFB3EFCB16B1E0DB06E104A5
:103D5000F10409F440C1C701B601F7DCEFEFCE1A58
:103D6000DE0AEE0AFE0A8111EECF0150A9CF8BEFD9
:103D7000820D833098F54601570153E0850E911C62
:103D8000A11CB11CC301B201E0DC8B838115E9F0F9
:103D9000C501B401DADC8C83811581F08B819C81B3
:103DA0008130AFEF9A0710F0982F8827B6E02B16D6
:103DB00079F0E7E02E1679F00E9426294601570196
:103DC000F4E08F0E911CA11CB11C750164017FCF22
:103DD0000E94C228F3CF0E94F428F0CFF4E05301F0
:103DE00042012F12F2CFC301B201AFDC782E46019F
:103DF000570124E0820E911CA11CB11CC701B60121
:103E00006D5F7F4F8F4F9F4FA0DC711409F4E3C0AB
:103E1000811509F4E0C08150990B4FEF489F900144
:103E2000499F300D1124472D4150550B240F351F4C
:103E30002150310950F28FE99FE00197F1F700C05E
:103E40000000F6CFC8013EDEC0CF6801A7E5DA1A50
:103E5000C114B1E0DB0608F45AC0ED81FE81958102
:103E60008091F4048272F801911509F4E3C0E052E4
:103E7000F847EB30F10508F008C1EB51FA4C0C940F
:103E8000B134C80197558115914038F7F801FF27E3
:103E9000053008F0A0C034E0EE0FFF1F3A95E1F7BF
:103EA000AF0141565B4F6A01AD81BE8115968C9181
:103EB000EC55FB4F908180FB90F99083811509F4BC
:103EC0006CC00E94510D9093F2048093F104F601AE
:103ED00082818F5F82838091F6049091F404892B14
:103EE00083838091F3048483468157816685778537
:103EF000C6010E94BE0CD60115968C9181FD4AC068
:103F0000902F812F9093EF048093F004A6CF65E962
:103F100074E08C2DF7DC892B09F0B8CFC60144E0A2
:103F2000880F991F4A95E1F7FC01E156FB4F22816A
:103F3000213029F52091950430919604232B09F422
:103F4000A5CF2091970430919804232B09F49ECF9C
:103F50002091990430919A0440919B0450919C04C3
:103F6000242B352B232B09F091CFFC01EC55FB4F73
:103F700020812E7F208381569B4FEADA87CF223023
:103F800009F084CF2091990430919A04232B09F4ED
:103F90007DCFEBCF90E080E0B5CFFA014485558529
:103FA00066857785C6010E94BE0CD60115968C9158
:103FB00081FF53CFC601B0DA8091EF049091F004F5
:103FC0000817190709F049CF1092F0041092EF0476
:103FD00044CF0E94290B8091F7048770811569F006
:103FE000AD81BE8115968C91811539F0809199052E
:103FF00082FF03C082E00E9481042696E2E10C94D5
:10400000DA34811559F10E94730BE5CF811559F10E
:104010000E94970BE0CF811559F10E94AC0BDBCFCA
:10402000811559F10E94C40BD6CF811559F10E9418
:10403000DA0BD1CFE054F847ED30F10530F5E0511F
:10404000FA4C0C94B1340E94330B81E00E94160BA1
:10405000C2CF0E94410BF9CF8115A9F20E94690BD2
:10406000BACF8115A9F20E948E0BB5CF8115A9F2A6
:104070000E94A00BB0CF8115A9F20E94B80BABCF64
:104080008115A9F20E94D00BA6CF0737FCE71F07C6
:10409000F9F008372CE7120731F19801205E32451C
:1040A0002032310528F591113AC00F7181E090E07E
:1040B0007C01002E02C0EE0CFF1C0A94E2F76E2D6C
:1040C00083E090E00E9469358E2D0E94D00383CF5B
:1040D00081E0911551F00E94D60343E062E081E057
:1040E0000E94580478CF82E0F4CF0E94E003F5CF1D
:1040F0009115A9F00A354CE7140709F478C008F0C7
:1041000050C001308CE7180709F46FC003309CE7FA
:10411000190709F464C001151C4709F453C0ED8167
:10412000FE8187819085009709F465C00E94A205F1
:104130008C01ED81FE81B580A680A2942FE0A222A1
:104140008091F7048770811501F1CB2CB114F1F047
:10415000812F807F803461F080E2800F8830A8F06A
:10416000812F807E803221F4023078F0A11469F032
:104170008091990582FF09C082E00E9481048091AC
:10418000F7048770CC24C3948111C12CE12FE295F0
:10419000EF70103C08F0A7C0F0E0E350FA4C0C942C
:1041A000B1340B35BCE71B0721F180919905002440
:1041B00082FF0394802D0C351C4709F0B0CF0E947C
:1041C000E415ADCF0E947D17FFEF24E34CE0F150E2
:1041D00020404040E1F700C000000E9459156FEFF9
:1041E0007FEF80E090E00E9483350E94AC1781E071
:1041F000E6CF80E0E4CFAD81BE8115968C91159716
:10420000CD90DC90811559F0C60114DAF82E682F94
:10421000C6010E94EE03B6018F2DF1D987CFC601EA
:104220000E942404F82EF7CFF12FFF70DF2E1031FB
:1042300018F0D29490EFD922B114B9F0D11469F0EA
:1042400080E2800F883010F0011109C08091F404E1
:104250008D298093F4040E942216802F42C0809101
:10426000F6048D298093F604F6CF802F0E9416174E
:10427000D114C9F180E2800F883010F0011104C020
:104280008D2D0E949C0406C0D0948091F6048D214F
:104290008093F6040E94221626C0212F2F70D22E62
:1042A000107F103219F0D29480EFD822011549F016
:1042B000013009F485C0B11409F491C0A114B9F119
:1042C000CCCF8091990582FD2EC0B11431F1D1146B
:1042D00039F08091F4048D298093F4040E94221611
:1042E00080E00E947816C11409F4D9C08091F704C7
:1042F00080FDD5C0ED81FE811582869586958695D7
:104300000E94D6038D819E8185DC8091F70486957D
:10431000869586950E94E003C2C080E00E94161731
:10432000D11409F3ADCFB11469F1A11004C08D2DE2
:104330000E945B17D8CF41E0A41210C0F090F304A4
:104340008D2D8F21D81679F20E94510D9093FB0488
:104350008093FA04FD28F092F304C5CF55E0A5122E
:10436000C2CF8D2D0E945B178D2D0E94AD0D8091C7
:10437000F5049D2D9823D91609F4B5CF8D29809386
:10438000F504B1CFA11012C08D2D0E9464178D2DA0
:104390000E94AD0D8091F5049D2D9823911509F48F
:1043A000A2CFD094D822D092F5049DCF81E0A8125C
:1043B0009ACF8091F4048D21811509F494CFE4CF34
:1043C000B11429F096E0A91608F08DCFB0CFA5E082
:1043D000AA1608F088CF8D2D0E94641784CFA114EF
:1043E000D1F3093349F4BFEFE7EEF3E0B150E04019
:1043F000F040E1F700C00000802F0E94161773CF35
:10440000812F869586958370811561F0813009F042
:104410006ACFC8019370B11002C080E090E00E94A2
:10442000FA0C61CFC8019370B11002C080E090E037
:104430000E94D20C58CF6B2D802F0E94EB0D53CFD2
:10444000812F8370811138C0B11027C0402F429551
:1044500046954770440F440F802F8F70042E01C083
:10446000880F0A94EAF7202F207104FF07C02FE07D
:1044700030E001C0220F4A95EAF72095169516956F
:1044800013701230A1F0133081F040919605113075
:1044900059F0822B84230E94D0030E94C30C60E059
:1044A0008D819E81F1D8A9CD842B822BF4CF822BD4
:1044B000909196058927EFCFB11451F110FFEDCF00
:1044C000402F429546954770440F440F802F8F70C0
:1044D000042E01C0880F0A94EAF7202F207104FFF0
:1044E00007C02FE030E001C0220F4A95EAF720957F
:1044F000169516951370123089F0133069F04091BB
:104500009705113041F0822B84230E94D303C5CF3D
:104510008230B0F6C2CF842B822BF7CF822B9091C2
:1045200097058927F2CF1F70B11439F0812F0E94AF
:10453000D603802F0E945B17B0CF802F0E94641794
:10454000812F0E94E003A9CF023F71F170F4003F78
:10455000C9F0013F91F0B11409F465C0A11409F448
:104560005FC0802F0E94781698CF033F21F1043F4F
:1045700091F78091990582FD2AC0812F8F71B11426
:1045800001F316C0B11469F025E0A21608F085CF3A
:104590001F7181E090E0012E01C0880F0A94EAF7B4
:1045A000BECF46E0A416F2CF812F8F71B110C9CFD4
:1045B0000E94D60372CF80E0B11409F4A6CF1F7118
:1045C00081E0012E01C0880F0A94EAF79ECFB11452
:1045D000C1F08091F7048770843049F41092F70499
:1045E0001092F9041092F804812F8F71AACF55E030
:1045F00063E0A51608F051CF812F8F710E94970DAF
:104600004CCF85E0A81640F01092F7041092F90400
:104610001092F80464E0F0CF81E00E9481043DCF65
:10462000812F8F71C5CFA114F9F2093349F49FEF9F
:10463000A7EEB3E09150A040B040E1F700C0000009
:10464000802F0E94161729CFA0E0B0E0EAE2F3E243
:104650000C94C93480917704803108F047C0809170
:104660007604811509F442C0C091280489E0D82E4F
:10467000809127048C17D1F1EC2EF12CDC9EE00107
:104680001124FE01E75DFB4F84818115A1F1918129
:104690008091720498132FC09081809171049813B7
:1046A0002AC08581811127C0028113818091730402
:1046B00090917404081B190B60E081E794E00E945C
:1046C000441B35D908171907B0F4809177048F700F
:1046D000806180937704C15DDB4F88818F7080613A
:1046E000888381E794E096DA0E947704CDB7DEB73D
:1046F000E7E00C94E534E7012196C770B9CFAFE04D
:10470000B0E0E5E8F3E20C94C1348C0186E0F801F6
:10471000DE011A9601900D928A95E1F7F801F58075
:10472000E48081E7882E84E0982E809175048111C1
:1047300017C0E11491F0F11409F479C1C8010E9485
:10474000731B811509F473C189E0F801A1E7B4E096
:1047500001900D928A95E1F777DFFF24F39468C00A
:10476000A280B380D09076048091730490917404F9
:104770003501681A790AD11409F40AC1C080518040
:1047800060E081E794E00E94441BD1D86816790666
:1047900008F0B2C0E11409F380917204F80191812C
:1047A000E0907704F0E1EF1608F062C098131FC0A4
:1047B00090917104F8018081981319C020917804B8
:1047C00030917904878190852817390781F4F11099
:1047D00049C08E2D8F7080618093770481E794E0CB
:1047E00019DA80917704F8018683F12C21C0F11049
:1047F00039C040E0652D8C2D0E94141540E0652DD8
:104800008C2D0E941415F82E8111EFCF8A859B857F
:104810000E94661B292F22952F70903470F49F7090
:10482000223098F09115A9F0F8019681903188F422
:104830008F2D2F96EFE00C94DD342A5F2F702230FD
:1048400060F0C801E7D9FD2CF3CF911511F0811567
:1048500079F3805E883060F3F4CF803F48F3815F66
:104860008330F9CF80917704816080937704BDCF46
:1048700098131DC090917104F8018081981317C09E
:104880002091780430917904878190852817390721
:1048900071F4F1100CC0E682C801BCD989E0F801BE
:1048A000A1E7B4E001900D928A95E1F756CFC801D7
:1048B0000E94731B811509F4BAC0F11409F4B7C042
:1048C00080917704803208F43FCF809171049091F9
:1048D00072049A838983BC82AB82809175048D8334
:1048E0001E82EF828091780490917904998788875D
:1048F000CE0101968FD928CFD0907704F0E1DF1652
:1049000048F481E794E086D989E0F40111928A9510
:10491000E9F76BCFE11409F420CF90917204F8010C
:104920008181981319C0909171048081981314C0EB
:104930002091780430917904878190852817390770
:1049400059F4F11009C0D682C80164D989E0F40194
:1049500011928A95E9F701CFC8010E94731B811556
:1049600009F465C0F11409F462C0809177048032C3
:1049700008F4EACE80917104909172049A8389833D
:10498000BC82AB82809175048D831E82DF82AACFA8
:1049900060E081E794E00E94441B0E94971C681627
:1049A000790608F0B1CFE11409F4D7CEF11409F477
:1049B0003EC090917204F801818198132EC09091AD
:1049C00071048081981329C0209178043091790472
:1049D000878190852817390701F58091730490919C
:1049E0007404A81AB90AF8ECAF16B10408F056CF4F
:1049F0008091770480FD52CF803108F44FCFF801C9
:104A00008683982F907F903F09F446CF982F907F10
:104A1000905F8F70892B86833FCFC8010E94731BE4
:104A2000811192CE80917704816080937704C801D0
:104A3000F1D893CEA2E1B0E0E0E2F5E20C94CC3400
:104A40000A871B872C873D874E875F87688B798B0A
:104A50008A8BCE010A9653DE811128C0209127044B
:104A60003091280489E0FE013A96DE01119601900A
:104A70000D928A95E1F78E858115C1F0822F90E025
:104A800001968770992738171906D9F099E0929FF7
:104A9000D0011124A75DBB4FFE01319601900D920C
:104AA0009A95E1F7809327040E94770419E080919A
:104AB000280490912704891312C06296E4E00C94B4
:104AC000E8340E947D17109227041092280489E090
:104AD000E1E7F4E0DF011D928A95E9F7E7CF189F3F
:104AE000C0011124875D9B4F0ADE811531F380914F
:104AF000280490E001968770992780932804D7CFE7
:104B0000EF92FF920F931F93CF93DF9380919305C2
:104B1000E091B602CDE0811130C0CDB7DEB7E6E05E
:104B20000C94E634D1E0DE0FD093B602EE2EF12CD9
:104B3000CE9FF0011124E55DFA4F84818115E1F0EB
:104B400087819085892B21F481859285019651F486
:104B50000081118122813381448155816681778171
:104B6000808568DFCE9DF001CF9DF00D1124E55DBD
:104B7000FA4F14821092F604ED2F80919305E817F6
:104B800088F2109293051092B602C7CFA4E0B0E06D
:104B9000ECECF5E20C94BF3420912A05298397E0D0
:104BA000992E01E010E02DE0322E34E0532E8824BF
:104BB0008394809129059981891307C0A1DF0E9400
:104BC0002E0C2496E1E10C94DB349981892F90E03E
:104BD0009C838B83FC01EE0FFF1FE15EFA4F808107
:104BE0009181989ED001999EB00D1124FD01E45051
:104BF000FB4FFA83E983248121115BC06090930508
:104C0000EBE2F5E060E070E0712C661508F04FC053
:104C1000A384B484A981BA81CD90DC902FEF3FEFBB
:104C2000412C442D50E07601E40CF11CE40CF11C05
:104C3000D701ED90FC90E114F10439F0AE14BF04FB
:104C400009F0A90143949A01ECCF2F3F3207D1F12B
:104C5000D80102C0AA0FBB1F2A95E2F77A2A980151
:104C6000042C02C0220F331F0A94E2F7A90141501D
:104C700051097416150629F5369EF001379EF00D80
:104C80001124E55DFA4F989ED001999EB00D112434
:104C9000A450BB4F12962D913C91139730872783D8
:104CA0005482108211829287818715968C920E947D
:104CB0003F0C8B819C8101969A83898383708983C1
:104CC00078CF14826F5F7F4F3D969FCF10929505EE
:104CD0001092940510921C018091290580932A0559
:104CE0000E942E0C0DCFACE1B0E0E9E7F6E20C94A7
:104CF000BE344B8B5C8B6D8B7E8B8F8BB92E988FDC
:104D0000A92E91111092F604188A198A1A8A86E03F
:104D1000FE017396DE011A9601900D928A95E1F7D5
:104D20005F888091990582FF1FC00E94510D2091DC
:104D3000F8043091F904821B930B8838934138F0C2
:104D40008091F70482FD03C082E00E9481040E94EA
:104D5000510D2091FA043091FB04821B930B88388B
:104D6000934110F00E94A4045114D9F05E86BF86CE
:104D700061E0CE010A960E94441B61E0CE010A96D2
:104D80000E94441B61E0CE010A960E94441B4C0124
:104D900080354CE7940791F4A11411F181E08093E0
:104DA0001C015E86BF860A851B852C853D85452DA9
:104DB0005B2D688979898A893DDECDC081355CE7C4
:104DC000950721F4A11461F081DFEBCF82359C4778
:104DD00039F4A11429F080911C018111F5CFDECFA7
:104DE0004CEFE42E44E0F42E412C612C712CD701C1
:104DF0006D917C91CC24CA94DD24DA9480E0282F34
:104E000030E0FB01E80FF11DE80FF11D40815181F9
:104E10004115510539F08416950609F096018F5F0A
:104E20006901EDCF10E0BFEFCB16DB0609F44FC0F0
:104E3000F701448110911C01411110E0D701159632
:104E40003C90159716962C911697A11409F406C15B
:104E5000111509F403C1311017C041E050E00C2CCA
:104E600001C0440F0A94EAF7242B16962C93209144
:104E70002705309128052233310530F422E330E054
:104E8000309328052093270521E030E0F90102C086
:104E9000EE0FFF1F8A95E2F7CF010197D701169613
:104EA0002C912817190699F4C0909405D090950577
:104EB000C114D10409F453C00E94510D8C199D09ED
:104EC000C39708F44CC081E0F701848311E0412AC4
:104ED000BFEF6B1A7B0AE7E0EE0EF11CF5E06F16F0
:104EE000710409F084CFA11409F416C1411409F426
:104EF00013C10E94510D9093950580939405809164
:104F00009305883040F591E0980F9093930599E0D0
:104F1000FE013A96DE01119601900D929A95E1F705
:104F20005D82BE822DE0829FC0011124855D9A4F73
:104F300029E0FE013196DC0101900D922A95E1F7FE
:104F40002FEF3FEFDC011A963C932E9319971C9696
:104F50009C928E921B976C96E2E10C94DA3420912D
:104F60002A0580912905922FE0E0F0E001E0281762
:104F700009F448C0A22FB0E0FD01EE0FFF1FE15E73
:104F8000FA4F2080318037E0329DF001339DF00DE3
:104F90001124E450FB4F408151815C8F4B8FC12C19
:104FA00030E0D12CEB8DFC8DED0DF11DED0DF11DE3
:104FB0004081518141155105E1F0F7010190F081E7
:104FC000E02DFA8FE98F30E007C0E1E04617570780
:104FD00009F0E0E0CE2A3F5FE98DFA8DE30FF11D85
:104FE000E30FF11D608171816115710571F7D39433
:104FF000D9CFC11481F13D15C8F421E0D701149631
:105000002C93F70190932A05EE15FF0509F45FCF65
:1050100090E0FC01EE0FFF1FE15EFA4F71826082AB
:105020000196837099278093290551CF37E0329DEF
:10503000F001339DF00D1124E450FB4F0483EE1575
:10504000FF05F9F2291302C09F5F93709D012F5F46
:105050003F4F23708CCFE0E0F0E0F8CF30E031102C
:1050600024C061E070E002C0660F771F8A95E2F706
:10507000CB0101972817390791F010E0E1E0F0E04B
:1050800002C0EE0FFF1FCA94E2F76F01C094D70170
:1050900016968C9116978C2116968C9318CF4115E5
:1050A00069F3C3010E943F0CE8CFA9010C2C02C098
:1050B000559547950A94E2F7C901019782239323F6
:1050C000892B39F540FF25C0D70112968D919C910F
:1050D000892BD1F087E0FE013196DF011D928A9580
:1050E000E9F70E94510D9C018B839C8384E08D83A2
:1050F000F70192818381792F9887898709811A81A5
:1051000044E05E816F8196DCD70115961C92132DC9
:10511000B5CF142F1170B2CF90912A058091290537
:10512000981731F033DDB1E04B1609F414CF39CEC6
:10513000E7DC10929505109294050E942E0CF3CF97
:10514000A6E0B0E0E6EAF8E20C94CC340E94510DFF
:105150008C018091FB039091FC038017910771F003
:1051600019821A820E94510DBC0149815A8180E046
:1051700090E0B9DD1093FC030093FB032696E4E076
:105180000C94E834A6E0B0E0E8ECF8E20C94CC34FF
:105190008C019093F8038093F703011580E21807C0
:1051A000B0F4C801805E9109089728F06AE677E1BB
:1051B0000115110511F46BE577E1C8010E94A40304
:1051C000802F0E9478162696E4E00C94E83480EF55
:1051D00089838A830E94510D8160BC0149815A8173
:1051E00081E091E080DDEFCFA6E0B0E0EAEFF8E209
:1051F0000C94CC348C019093F8038093F703011541
:1052000080E21807B0F4802F0E941617C801805E54
:105210009109089728F063E777E10115110511F46A
:1052200064E677E1C8010E94A4032696E4E00C94AA
:10523000E83480EF89838A830E94510D8160BC012C
:1052400049815A8181E090E04EDDEFCFCF93DF932B
:10525000D82FC92F97DF8D2F9C2FC6DFDF91CF91DD
:1052600008950F931F93CF93DF938C01862F65E9E9
:1052700074E00E94821C892B91F4C0919504D09116
:105280009604209761F0F8018281833039F4CE01D1
:10529000DDDFCE01DBDFCE01D9DF01C0E0F7DF913A
:1052A000CF911F910F9108950F931F93CF93DF9389
:1052B0008C01EB0165E974E08C2F0E94821C892B24
:1052C00009F057C0FE01FF27D80112968C91129762
:1052D000E959FC4F8130A9F415968C9182FD4EC09E
:1052E00080FF4CC082E08083809197049091980465
:1052F0000097B9F480919504909196040097C9F1B4
:1053000010C08230A1F515968C9182FD26C080FDDB
:105310000AC083E080838091990490919A04009759
:10532000F1F030DF26C084E0808380919B0490916F
:105330009C040097B1F78091950490919604009792
:1053400001F184DF8091970490919804009749F7C8
:105350008091950490919604E4CF85E080838091BC
:10536000950490919604009721F070DFF1CF86E0CC
:105370008083DF91CF911F910F91089581E0808309
:10538000B9CF8091970490919804B8CF0F931F9351
:10539000CF93DF938C01EB0165E974E08C2F0E94C1
:1053A000821C892B71F4DD27C959DC4F8881F801F3
:1053B000128218828330E9F048F4813059F082304B
:1053C00081F0DF91CF911F910F9108958430B1F05A
:1053D0008530B9F78091950490919604009789F3F0
:1053E00006C08091970490919804009799F3FCDE91
:1053F000E8CF8091990490919A04F7CF80919B0413
:1054000090919C04009799F720919504309196040F
:10541000809197049091980421153105F9F2009735
:1054200031F7C901E4CF48E050E067E170E084EE75
:1054300093E00E945A3510927C030895E4EEF3E065
:1054400085E3808380911D0190911E01A0911F0131
:1054500081839283A3838FE784838FEF8583E3CF58
:105460004F925F926F927F928F929F92AF92BF9274
:10547000CF92DF92EF92FF92C0906C03D0906D03B9
:10548000E0906E03F0906F030E94A60E2B013C018A
:10549000530142018C189D08AE08BF080E94A60E59
:1054A000282F60936C0370936D0380936E03909329
:1054B0006F03A091A903E9EAF3E08A2F30E04FEFF0
:1054C000C40ED41EE11CF11CC418D508E608F70868
:1054D000A3132DC08093A9038091A703811137C026
:1054E0003091E403832F8370811519F0832F869503
:1054F0008695309115013230F1F158F5311138C0EF
:1055000010920401609370037093710320937203EF
:105510009093730389E2E9EAF3E0ADE7B3E0019029
:105520000D928A95E1F781E08093150114C0418DB9
:10553000528DC416D506E104F10420F481503F5F7A
:105540003296C6CF480D591D528F418FF8CF80E05B
:10555000D0CF3330D9F0FF90EF90DF90CF90BF9055
:10556000AF909F908F907F906F905F904F90089535
:105570000E944812F0CF809317018091E40383705A
:10558000809316010E94331583E0CECF80917C0377
:10559000811149DFC0907003D0907103E0907203D5
:1055A000F09073030E94A60E6C197D098E099F0965
:1055B000603171058105910570F210921501CBCF14
:1055C000A0E1B0E0E6EEFAE20C94C034FE013196C0
:1055D00080E1DF011D928A95E9F700E210E09DE08D
:1055E000A92E92E0B92E23EF422E55245394612C1C
:1055F000712C4F0173016201B1E14B16510461043A
:1056000071041CF080E1C82ED12CA601B501C401A3
:105610000E945A35AC0CBD1C0D2C000CEE08FF0886
:105620004C185D086E087F080150104019F760960D
:10563000E0E10C94DC346FEF85E290E00E94693584
:105640006FEF86E290E00E9469356FEF87E290E0AD
:105650000E94693560E088E290E00E9469350E940E
:10566000CF1BAEDF60ED85E290E00E94693569E511
:1056700086E290E00E94693569E287E290E00C944E
:105680006935CDB7DEB7E3970FB6F894DEBF0FBE2E
:10569000CDBF85B7806885BF85B7806885BF84B773
:1056A000877F84BF0FB6F894A895809160008861C9
:1056B00080936000109260000FBE80E890E00FB60B
:1056C000F89480936100909361000FBE81E0809315
:1056D0001B018EE996E090936F0280936E020E9408
:1056E000F10B0E943E1C0E945B0F0E94BA14809135
:1056F000E20084608093E20078948091F603811543
:1057000099F08091E9001091EC008F7017951127A6
:105710001795182B1092E9008091E80083FD0E94F4
:10572000C1171F701093E90082E084BD93E095BD1E
:105730009AEF97BD80936E000E94B61B811101C045
:105740007ADF85E90E94A00686E60E94A00686E32D
:105750000E94A00686EC0E94A00604E411E070E519
:10576000E72E71E0F72ED8018D918D018F3F11F05A
:105770000E94A006E016F106B1F788E0ECEEF3E037
:10578000DF01282F1D922A95E9F7E4E7F3E0DF0116
:105790001D928A95E9F780E090E00E945535833E9E
:1057A0009E4F21F40E94B61B81112AC063EE7EEF4A
:1057B00080E090E00E94833560E082E090E00E940B
:1057C000693581E08093960561E083E090E00E9476
:1057D000693560E074E184E090E00E9483352EDE5C
:1057E0002ADF40E050E0BA018FE090E00E947B3574
:1057F00040E050E0BA0183E190E00E947B3513DE87
:1058000082E090E00E944D358093D20384E090E0E6
:105810000E94553590939905809398050E94B21C7B
:10582000EFEFF6E721E0E150F0402040E1F700C063
:1058300000000E94B21C8091EC0380FF08C06FEF53
:105840007FEF80E090E00E9483350E94591583E04D
:1058500090E00E944D350E94D0030E94090C1092E6
:105860007D0340E150E06FEF70E086E993E00E9435
:1058700036351092A90340E150E06FEF70E082EC02
:1058800093E00E94363581E080937C0348E050E04D
:1058900067E170E084EE93E00E943D3510927C0356
:1058A0008091E403843008F4C9DD80919805806814
:1058B00080939805609198057091990584E090E037
:1058C0000E94833589E091E090931E0480931D042B
:1058D0008091F603853089F410E403E050E1F52E61
:1058E00062E1E62E8091F603853009F4DDC00E9466
:1058F0007D170E94C30C1092A7030E94B21CE3ED17
:10590000F3E0FEA7EDA74CEE842E43E0942ED401E5
:10591000219131918D919D9143E0EB3DF40709F484
:105920000FC128173907A1F330E5432E31E0532E7C
:105930008CEE93E098AB8FA71BA6AFA5B8A9ED900E
:10594000FD90B8ABAFA7EDA5FEA581919191FEA703
:10595000EDA78E159F0509F49BC09C012E253F25C0
:105960003BAB2AAB1201612CCC24C394D12C8AA965
:105970009BA98C219D21892B09F47DC086010E21D4
:105980001F2169823BA53A830E94510D9C838B8322
:1059900041E04D8391E00115110509F490E09E83EB
:1059A00049815A816B817C818D819DD9012B29F0A0
:1059B000D1018C918F3F09F033C2712C072D10E07B
:1059C0008091A903870D9927991F09976CF1B8E079
:1059D000AB2EB12CA01AB10AB80166557C4FA501B7
:1059E0008AEA93E00E942D35B8016E547C4FA501E0
:1059F00082EB93E00E942D35A501440F551FB8019D
:105A0000660F771F6E537C4F82EC93E00E942D351A
:105A1000B80166547C4FA5018AEB93E00E942D35B6
:105A200088E087198093A903711429F14091A90393
:105A3000B9A98B2F90E0242F30E0F901E755FC4FF6
:105A4000DC01AA0FBB1FA058BE4F5C915183880F89
:105A5000991FDC01A05BBE4FD1968C91818789A9EB
:105A6000818BF901EE0FFF1FE755FC4F128E118E4F
:105A70004F5F4093A9036394CC0CDD1C9FEF291A60
:105A8000390AACE06A1273CFEDA5FEA5F292E2925C
:105A9000BBA5BF5FBBA7ECE04E0E511CB43009F0B4
:105AA0004CCF0E94A60E51C08091F603843009F4B9
:105AB00038C0D6DC8091A70381110DC00E94481226
:105AC000109217018091E4038370809316010E9465
:105AD00033150093150131E03093A7031092A6030C
:105AE00088E190E00FB6F894A895809360000FBE0F
:105AF0001093600083B7817F846083BF83B7816028
:105B000083BF7894889583B78E7F83BF0FB6F89450
:105B1000A895809160008861809360001092600079
:105B20000FBE0E94B21CECEEF3E081919191892BA3
:105B300009F03BC5A4EFB3E0AE17BF07B1F7D2CE73
:105B40002817390709F0F0CEFBDAE090EF04F09067
:105B5000F004E114F10429F1C090F104D090F204B2
:105B60000E94510D8C010C191D09C7010E94971C40
:105B700080179107B0F42091EF043091F004C9012F
:105B80009927253008F050C144E0880F991F4A95A5
:105B9000E1F781569B4FDC0115962C9122FF0E9464
:105BA000A81A80911C01811519F10091940510919A
:105BB000950501151105E1F00E94510D801B910B17
:105BC00020912705309128052817390788F49091EE
:105BD0002A0580912905981709F429C10E94C62534
:105BE00010922805109227051092950510929405A1
:105BF00037DC86E0EFE8F4E0DE01119601900D92CB
:105C00008A95E1F7B0909004D090910400919204AD
:105C1000C0909304109194041092910410929204F5
:105C20001092930410929404802F8D29811509F409
:105C300041C0E090DD03F090DE030E94510D9C0115
:105C40002E193F0990918D04911509F4A9C42531AD
:105C5000310580F19F3F19F09F5F90938D04D1141F
:105C600059F00E94790C91E01D140CF09FEF899F70
:105C7000802D112480939104011559F00E94790C14
:105C800091E010160CF09FEF899F802D11248093D6
:105C9000920480919104811569F0F0909204F114BE
:105CA00049F00E946B0C809391048F2D0E946B0C25
:105CB00080939204812F8C29811509F441C0E090D2
:105CC000DB03F090DC030E94510D9C012E193F096B
:105CD00090918C04911509F45EC42135310580F151
:105CE0009F3F19F09F5F90938C04C11459F00E945C
:105CF000990C91E01C140CF09FEF899F802D1124CA
:105D000080939304111559F00E94990C91E011169B
:105D10000CF09FEF899F802D112480939404809133
:105D20009304811569F0F0909404F11449F00E94F5
:105D30006B0C809393048F2D0E946B0C80939404C2
:105D400080919004B81219C080919104811511F0CE
:105D50008D1113C020919204211511F002130DC072
:105D600090919404911511F0191307C03091930488
:105D7000311103C0822B892B81110E94C20D86E054
:105D8000FE013196AFE8B4E001900D928A95E1F7FB
:105D90000E94C30C9091DF03891721F08093DF03E9
:105DA0000E94A60E8091F603843009F091CD83E025
:105DB0008093E9008091E80082FF8ACD8091E8001D
:105DC00090E085FF0BC00E942A0F30E2E32EF12CF9
:105DD0008E010F5F1F4F8115E1F191E08091E80086
:105DE0008B778093E800911509F472CD0091F90347
:105DF0001091FA03E98101151105C9F1EE3F09F08F
:105E000058C08A81833020F08550833008F051C01B
:105E1000EA81EE3008F04DC0F0E0E75FF94CA1C533
:105E200089AB77247394CACD80E090E0B4CE0E9411
:105E3000802510929505109294050E942E0CD8CEC4
:105E40008091F100F80181938F01F1E0EF1AF108E0
:105E500021F28091E80085FDF3CF8091E8008B77F7
:105E60008093E8000E942A0F811599F3B6CFE431A0
:105E700048F4E11549F0E150E33130F4F0E0E95E37
:105E8000F94C6FC5EE3F21F28FEF898312C01A8261
:105E900089E08B830EC08A81823081F08330B1F03B
:105EA000813091F70E94A60E62D56B837C838D832F
:105EB0009E83CE0101960E947A0F0ACD88E290E07F
:105EC000ECD51B821C821D828E83F3CF8091F4035C
:105ED0009091F503892B69F3FE01319684EF93E0ED
:105EE000D4012C9111963C91B2E08B0E911C32831F
:105EF000238332968815990599F7DBCF8A81823002
:105F000019F66B817C818D819E8131D588E290E08C
:105F1000E0D5CFCF4C816B818A810E94D01A98271F
:105F2000892798279E838D83C4CF2D813E81322778
:105F3000232732274C816B818A810E94FB15B9CFC0
:105F40000E94CF1BB6CF8A81823831F178F4803835
:105F5000B1F0813809F0ADCF60E08B810E944D0B2C
:105F60008B81811116C00E94410BA3CF833809F0A9
:105F7000A0CF8B8120E04091E7036C8106C0809127
:105F8000E50320E04B816091E60390E00E947C0BEA
:105F900090CF0E94330B8DCFEB818FE7E43020F45C
:105FA000F0E0E250FE4F80818093E80380E00E94A1
:105FB000160B7FCF8A818238C1F050F4803891F07F
:105FC000813809F076CF8091E4038695869561CF7C
:105FD000833809F06ECF8091E5038B838091E603CF
:105FE0008C8367CF8091E70354CF8091E803873299
:105FF00030F08F3530F08E3930F482E04ACF80E0D7
:1060000048CF81E046CF83E044CF0DDA52CF85E020
:106010008A834FCF81E08A8383EF3BCF8C818D31A0
:1060200008F047CF8A809B80982489249824A12C4B
:10603000B12CFE0131967F018F01080F111D0E1545
:106040001F0509F436CF80E0F3EF8F16F1E09F06CD
:10605000A104B10420F4C401835F9D4F1ED5D70174
:1060600014968C93BFEFEB1AFB0AEFEF8E1A9E0A81
:10607000AE0ABE0AE4CF8091F4039091F503892B18
:1060800009F417CF8C818D3108F013CF882E912C15
:10609000A12CB12CCA80DB80DC24CD24DC24E12CB3
:1060A000F12C8E010F5F1F4F412C512C32014814EF
:1060B00059046A047B0408F0FCCEF3EFCF16F1E03C
:1060C000DF06E104F10438F4D80114966C91C6019E
:1060D000835F9D4FFED4BFEF4B1A5B0A6B0A7B0AAE
:1060E000EFEFCE1ADE0AEE0AFE0A0F5F1F4FDFCF78
:1060F00067DADFCE84E08CCF8C818D3108F0D9CE89
:10610000882E912CA12CB12CCA80DB80DC24CD24DC
:10611000DC24E12CF12C412C512C32018E010B5F3F
:106120001F4F481459046A047B0408F0C2CE80E073
:10613000F0E8CF16F1E0DF06E104F10418F4C6013F
:106140008996ABD4D8018D938D01BFEF4B1A5B0AB2
:106150006B0A7B0AEFEFCE1ADE0AEE0AFE0AE1CFE7
:106160002C81022F10E02D3108F0A3CE8A819B8173
:106170009827892798272C01612C712C8038F1E011
:106180009F0708F096CE822E912CA12CB12C40E8CE
:1061900051E060E070E0441955096609770942173B
:1061A00051056105710508F484CE2091F403309106
:1061B000F503232B09F03EC01C0129E2220E311CFD
:1061C00080FBEE24FF24E0F880FF0BC0889665D4A6
:1061D0009D8189279827892781159C4711F48FEF86
:1061E0008D83D501C401840D951DA61DB71D80FFAB
:1061F00019C0680141E0C41AD108CE0105968C0D82
:106200009D1D9CA78BA7C101800F911F46D4ABA5F4
:10621000BCA59C9181159C4721F48FEFEBA5FCA5B3
:1062200080838601FE013196EE0DFF1D2FEFE016F3
:10623000F10638F08E010F5F1F4FC12CD12C760173
:1062400025C09481858181159C4711F42483258381
:1062500042E0E40EF11C3296EACF80E8481681E075
:1062600058066104710430F4D80114966C91C2018F
:1062700089962FD4BFEFCB1ADB0AEB0AFB0AEFEFAC
:106280004E1A5E0A6E0A7E0A0F5F1F4FC814D904A9
:10629000EA04FB0410F30DCE8091F4039091F50312
:1062A000892B09F406CECE0101960E947A0FFFEFEA
:1062B00021EE34E0F15020403040E1F700C0000012
:1062C000C4CA88E0E0E2F1E0DE01919601900D920F
:1062D0008A95E1F7FE0132968FE1DF011D928A95E2
:1062E000E9F786E0898388E07F96DE0115960190C4
:1062F0000D928A95E1F7DDCD84E2898381E08A837E
:106300001B821C82D6CD8B819C81092E000CAA0B8E
:10631000BB0B25E0880F991FAA1FBB1F2A95D1F739
:10632000AC01BD01405E5F4F6F4F7F4F481759076B
:106330006A077B0708F4BDCD8432E1E09E07A10522
:10634000B10508F0B6CD4532F1E05F076105710592
:1063500020F044E251E060E070E0481B590BBC01C2
:106360006F547A4FCE01019662D3A3CD4AE150E03B
:106370006FEF70E0CE01079679D38091F4038983A3
:106380000A831B821C8281E08D838BE09DCD81E09E
:1063900090E09093FA038093F90382E390E0909366
:1063A000E3038093E2030E94510D9093E1038093F5
:1063B000E0037FCD0115110581F1D090EC03C09071
:1063C000EF03E090E003F090E1030E94510D8E197D
:1063D0009F098536910540F1C3FE26C0D0FE24C03A
:1063E0000E94510D9093E1038093E0038091E203BA
:1063F0009091E30301979093E3038093E203892B49
:1064000061F41092FA031092F90381E090E0909306
:10641000F5038093F40300E010E08091F403898396
:106420000A838091E20335CD82E390E09093E30309
:106430008093E203F2CF1092F5031092F40339CD6A
:1064400040E250E06FEF70E0CE0101960FD331CD06
:106450008B81823009F44DC060F4811133C0FE019C
:1064600033968EE1DF011D928A95E9F785E08983F5
:10647000CFCD833009F472C0843009F01ACD1C816D
:106480008AE0FE013596DE01919601900D928A9583
:10649000E1F789A59AA50E94E40B9AA789A78FEF37
:1064A000153060F4FAE01F9FB001112465527E4F51
:1064B0004AE050E0CE0181962AD380E089830E9491
:1064C0003E1CF7CC8C819AE0F92E8E010F5D1F4F98
:1064D000F8012F2D11922A95E9F7B8010E94821C2C
:1064E0008983F801DE01129601900D92FA94E1F78A
:1064F000E0CC1C818AE0FE013596DE019196019088
:106500000D928A95E1F789A19AA10E94E40B9AA3C2
:1065100089A38BA19CA10E94E40B9CA38BA38DA1BA
:106520009EA10E94E40B9EA38DA38FA198A50E941B
:10653000E40B98A78FA38FEF153060F43AE0139F18
:10654000B001112467557E4F4AE050E0CE0181969C
:10655000DED280E089830E94F10BABCC2C816AE013
:10656000CE018196DC01E62F1D92EA95E9F72530F0
:1065700080F4629FB001112465527E4F4AE050E0E2
:106580007CD280E089838AE0FE01B196DE0112961A
:10659000AECE8FEFF7CF2B30310508F0A3CBD0CBA9
:1065A0002B30310508F058CB85CB8091A80381159D
:1065B00009F498C9F9BCE9BC09B400FEFDCF80918B
:1065C000D8008F7D8093D8008091E0008260809316
:1065D000E0008091E00081FDFCCF0E947D1782C920
:1065E0001F921FB61F9211248F939F93AF93BF9357
:1065F0008091A603811113C08091AE029091AF02E9
:10660000A091B002B091B1024196A11DB11D80933D
:10661000AE029093AF02A093B002B093B102BF91CB
:10662000AF919F918F911F901FBE1F9018957894E6
:106630001F921FB61F9211248F939F93AF93BF9306
:106640008091AE029091AF02A091B002B091B102E0
:106650000196A11DB11D8093AE029093AF02A0934D
:10666000B002B093B102BF91AF919F918F911F90F3
:106670001FBE1F9018951F920F920FB60F921124F4
:106680002F933F934F935F936F937F938F939F933A
:10669000AF93BF93EF93FF938091E10082FF09C016
:1066A0008091E20082FF05C08091E1008B7F8093A2
:1066B000E1008091DA0080FF24C08091D80080FF43
:1066C00020C08091DA008E7F8093DA008091D9001B
:1066D00080FFA9C080E189BD82E189BD09B400FEC7
:1066E000FDCF81E08093F60380919D02811109C066
:1066F0000E945B0F0E94BA148091E2008460809334
:10670000E2008091E10080FF1AC08091E20080FFEA
:1067100016C08091E2008E7F8093E2008091E200BB
:1067200080618093E2008091D80080628093D800DD
:1067300019BC85E08093F60383E080931B01809170
:10674000E10084FF2FC08091E20084FF2BC080E134
:1067500089BD82E189BD09B400FEFDCF8091D800DA
:106760008F7D8093D8008091E1008F7E8093E1003F
:106770008091E2008F7E8093E2008091E200816050
:106780008093E20080919C02811509F452C084E05C
:106790008093F6038091F603843009F052C082E0C2
:1067A00080931B018091E10083FF2CC08091E20067
:1067B00083FF28C08091E100877F8093E10082E021
:1067C0008093F60310929C028091E1008E7F80936B
:1067D000E1008091E2008E7F8093E2008091E200F0
:1067E00080618093E20042E060E080E00E948A14D1
:1067F0008091F00088608093F00081E080931B011D
:1068000080931A01FF91EF91BF91AF919F918F916A
:106810007F916F915F914F913F912F910F900FBE9C
:106820000F901F90189519BC1092F60310929D02BC
:1068300068CF8091E30087FF02C083E0A9CF81E0A9
:10684000A7CF81E0ADCF1F920F920FB60F92112408
:10685000EF92FF920F931F932F933F934F935F936A
:106860006F937F938F939F93AF93BF93CF93EF9348
:10687000FF9309EE10E0F8018081C091EC008F7069
:10688000C795CC27C795C82B108280EFE82EF12C36
:10689000F7018081877F808378940E94C117F80177
:1068A0001082F701808188608083CF70F801C083F7
:1068B000FF91EF91CF91BF91AF919F918F917F9178
:1068C0006F915F914F913F912F911F910F91FF9089
:1068D000EF900F900FBE0F901F901895AA1BBB1B37
:1068E00051E107C0AA1FBB1FA617B70710F0A61BD0
:1068F000B70B881F991F5A95A9F780959095BC01F1
:10690000CD01089597FB072E16F4009406D077FD6D
:1069100008D0E4DF07FC05D03EF4909581959F4FA9
:106920000895709561957F4F0895052E97FB16F495
:1069300000940FD057FD05D058D007FC02D046F484
:1069400008C050954095309521953F4F4F4F5F4F70
:10695000089590958095709561957F4F8F4F9F4FCB
:106960000895EE0FFF1F0590F491E02D099469271B
:106970009627692778278727782708952F923F92AF
:106980004F925F926F927F928F929F92AF92BF923F
:10699000CF92DF92EF92FF920F931F93CF93DF93EB
:1069A000CDB7DEB7CA1BDB0B0FB6F894DEBF0FBE48
:1069B000CDBF09942A88398848885F846E847D8495
:1069C0008C849B84AA84B984C884DF80EE80FD8097
:1069D0000C811B81AA81B981CE0FD11D0FB6F8940D
:1069E000DEBF0FBECDBFED010895A1E21A2EAA1B96
:1069F000BB1BFD010DC0AA1FBB1FEE1FFF1FA2176F
:106A0000B307E407F50720F0A21BB30BE40BF50B6B
:106A1000661F771F881F991F1A9469F760957095F4
:106A2000809590959B01AC01BD01CF010895FB01BC
:106A3000DC0102C005900D9241505040D8F70895F6
:106A4000FB01DC0104C08D910190801921F44150BB
:106A50005040C8F7881B990B0895FB01DC0102C068
:106A600001900D9241505040D8F70895DC0101C0CB
:106A70006D9341505040E0F70895DC01CB01FC01DB
:106A8000F999FECF06C0F2BDE1BDF89A319600B487
:106A90000D9241505040B8F70895F999FECF92BD3C
:106AA00081BDF89A992780B50895A8E1B0E042E049
:106AB00050E0E5CFDC01A40FB51F4150504040F03D
:106AC000CB01840F951F2E9105D041505040D8F72F
:106AD0000895262FF999FECF92BD81BDF89A0197AE
:106AE00000B4021639F01FBA20BD0FB6F894FA9A16
:106AF000F99A0FBE08950396272FECDFEADF252FC2
:106B0000E9DF242FE7CF0196272FE4DFE2CFDC0176
:106B1000CB0102C02D9105D041505040D8F70895C7
:106B2000262FF999FECF1FBA92BD81BD20BD0FB6A9
:106B3000F894FA9AF99A0FBE01960895F894FFCF47
:106B4000F70DFC0DFE0D030E130E130E130E130E98
:106B5000130E130E130E130E050E090E0C0E110E4E
:106B6000210E270E2B0E76128012A812E6121B138E
:106B700055137013731376137A137D1381138413D3
:106B800087138A138D1390139313961399139C13E1
:106B9000A013A313A613ED133214351438143B14A9
:106BA0003F1442144E1452145D1460146B146E148E
:106BB00079147C148714A218C818CE18C818CE18D7
:106BC00021194319CE184A1A571AE91F01202C20FF
:106BD000062031200B20362010203B20152040209D
:106BE00023202920E91F01202C20062031200B2002
:106BF000362010203B2015204020142114214D2147
:106C00004D2100221B227321732120229322A422D2
:106C1000A42261317C318331592F592FB631C731CC
:106C2000DA311B322032592F592F592F2832472F52
:106C30004B2F7E2F8A2F952FA02FA32FDA2F0530D1
:106C4000442F4C3107300A300E303B3078307A30E8
:046C50007C30B030B4
:106C54002B002B0000FF0039054E0DBF15D515DAAA
:106C640015DF15B61503FFFF000001000100FFB496
:106C74003C60D733A9A417B9004422B68401620149
:106C8400AC008A02A302C302003131295A1B750ADF
:106C9400956636C6349796943567F0F7F6F1F4F5B1
:106CA400292827262524232221201F1E1D1C1B1AC8
:106CB400191817161514FF131211100F0E0D0C0BC3
:106CC4000AFF090807060504FFFF03FFFF0201008E
:106CD400E040CC40B7408740544030401940034026
:106CE400E02BCC2BB52B9E2B892B752B612B4C2B9E
:106CF400382B242B082BD815BC15A81594157F15F3
:106D04006B15571542152E1519150315E000CC0007
:106D1400B700A3008F007A00660051003D002900EF
:106D2400140000000404040404040404040404011E
:106D34000101010101010404010101010101010139
:106D440001040401010101010101010101040F3FDA
:106D54007FBDE200E900EA00B500B600B700CD004F
:106D64008301CC008A0192019401210223022402AE
:106D74002502260227022A02B300B4006F00700025
:106D84009F01CB019F02A002E200E900EA00B500E6
:106D9400B600B700CD008301CC008A0192019401B2
:106DA4002102230224022502260227022A02B3001A
:0E6DB400B4006F0070009F01CB019F02A0028F
:00000001FF
